:100000000C9434000C9451000C9451000C94510049
:100010000C9451000C9451000C9451000C9451001C
:100020000C9451000C9451000C9451000C9451000C
:100030000C9451000C9451000C9451000C945100FC
:100040000C9451000C9451000C9451000C945100EC
:100050000C9451000C9451000C9451000C945100DC
:100060000C9451000C94510011241FBECFEFD8E026
:10007000DEBFCDBF13E0A0E0B1E0E6EAFFE802C0DA
:1000800005900D92A636B107D9F723E0A6E6B3E0B6
:1000900001C01D92AF38B207E1F70E9454000C94E2
:1000A000D1470C94000008950E9458000E94AF4769
:1000B0002F923F924F925F926F927F928F929F9278
:1000C000AF92BF92CF92DF92EF92FF920F931F9366
:1000D000CF93DF93CDB7DEB7CF50D1400FB6F894B2
:1000E000DEBF0FBECDBF8FB7F89490918E039030D6
:1000F00009F09BC391E090938E038FBF2D98259AB2
:100100005998519A8FEC90E09093C5008093C40069
:1001100082E08093C00088E18093C10086E08093F4
:10012000C2002D9A8E01095F1F4FC8014C9640E412
:1001300050E05C01612D0E94CA47C801089662E543
:1001400073E044E150E04C010E94C147045A1F4F44
:1001500080E090E07801F801828393833F010FB63D
:10016000A5968EAF9FAFA5970FBE8D879E878B8775
:100170009C8789879A878F8398878C0168E371E0D1
:100180004AE050E06501C5015A010E94C147F301F0
:10019000028313830FB6A596AEAEBFAEA5970FBE72
:1001A0008091C0008072803009F444C380E4809361
:1001B000C6008091C00080728030D9F388E48093BB
:1001C000C6008091C00080728030D9F38FE68093A2
:1001D000C6008091C00080728030D9F38CE6809395
:1001E000C6008091C00080728030D9F381E6809390
:1001F000C6008091C00080728030D9F380E2809385
:10020000C6008091C00080728030D9F38DE6809363
:10021000C6008091C00080728030D9F385E780935A
:10022000C6008091C00080728030D9F38EE6809342
:10023000C6008091C00080728030D9F384E680933C
:10024000C6008091C00080728030D9F38FE6809321
:10025000C600CE0185589F4F44E150E0B4010E9492
:10026000C147F701E280F380A080B1806D847E8475
:100270004B845C8429843A840F811885CE01815790
:100280009F4F40E850E08D839E83612D0E94CA47B6
:10029000D101B2019301A501040F151FAE1DBF1DB1
:1002A00080E090E05C016A1D7B1D2A1D3B1D4138EA
:1002B000510508F0C8C24134510508F0C6C2CB014F
:1002C000892F82958F7099278695220F331F220FD1
:1002D000331F220F331F282B392BF901FE2FEE2756
:1002E000CD01892F82958F7099278695660F771F8C
:1002F000660F771F660F771F682B792BCB01892F2D
:100300009927EB83FC838E2B9F2B89839A83762FEF
:100310006627C801892F82958F7099278695AA0F25
:10032000BB1FAA0FBB1FAA0FBB1FA82BB92BCD0148
:10033000892F9927862B972B2C01BA2FAA27C80122
:10034000929582958F7089279F70892796958795BA
:1003500090708A2B9B2B1C01232F3327ED80FE806E
:10036000C7015B01B60169013D014A010E94C14715
:10037000D7019401A20FB31F80E88C932833C201E8
:10038000310508F038C09070682A792A0FB6C35733
:10039000DF4F6EAE7FAECD58D0400FBE89819A81BF
:1003A0009070A82AB92A0FB6C557DF4FAEAEBFAEC0
:1003B000CB58D0400FBE4B805C804C285D280FB6D8
:1003C000C757DF4F4EAE5FAEC958D0400FBEC10118
:1003D0009070102F0027110F110F110F082B192BE0
:1003E0000FB6C157DF4F0EAF1FAFCF58D0400FBE73
:1003F000BE0161572FC09070682A792AF701E8582A
:10040000FF4F6482758289819A819070A82AB92AE7
:10041000A282B382C1019070102F0027110F110F1B
:10042000110F082B192B068317834B805C804C28F7
:100430005D280FB6C753DF4F4EAE5FAEC95CD040EC
:100440000FBECE0185589F4FB7010E9447106D81A6
:100450007E81605C7F4FCE0185589F4F0E94471080
:100460000FB6C35BDF4F8EAD9FADCD54D0400FBEF6
:100470000FB6EC968EAFEC970FBE0FB6EB969EAF15
:10048000EB970FBE0FB6C15BDF4F8EAD9FADCF5464
:10049000D0400FBE0FB6EA968EAFEA970FBE0FB6EA
:1004A000E9969EAFE9970FBE0FB6C75BDF4F8EADE3
:1004B0009FADC954D0400FBE0FB6E8968EAFE897F7
:1004C0000FBE0FB6E7969EAFE7970FBE0FB6C55BA0
:1004D000DF4F8EAD9FADCB54D0400FBE0FB6E6962A
:1004E0008EAFE6970FBE0FB6E5969EAFE5970FBEAF
:1004F0000FB6CB5BDF4F8EAD9FADC554D0400FBE66
:100500000FB6E4968EAFE4970FBE0FB6E3969EAF9C
:10051000E3970FBE0FB6C95BDF4F8EAD9FADC754DB
:10052000D0400FBE0FB6E2968EAFE2970FBE0FB669
:10053000E1969EAFE1970FBE0FB6CF5BDF4F8EAD5A
:100540009FADC154D0400FBE0FB6E0968EAFE0977E
:100550000FBE0FB6AF969EAFAF970FBE0FB6CD5B77
:10056000DF4F8EAD9FADC354D0400FBE0FB6AE96D9
:100570008EAFAE970FBE0FB6AD969EAFAD970FBEC6
:100580000FB6ED968EAD9FADED970FBE0FB6AC9644
:100590008EAFAC970FBE0FB6AB969EAFAB970FBEAC
:1005A0000FB6EF968EAD9FADEF970FBE0FB6AA9622
:1005B0008EAFAA970FBE0FB6A9969EAFA9970FBE92
:1005C00080E090E09E0129593F4FD901A80FB91F43
:1005D0004C91542F52955F70A52FBB27A85DBE4F3D
:1005E0005C91DC01AA0FBB1FFD01EA59FC4F50834F
:1005F0004F70E42FFF27E85DFE4F4081A959BC4FA3
:100600004C9301968431910501F700E010E027E654
:1006100033E02E7F46E653E0241B350B4FEFF80105
:10062000DF01AA59BC4F5C91652F66230AF431C0E3
:100630002F3F340709F4BCC0B9016E1B7F0B6170FA
:1006400070706030710509F0B3C0E532F105BF018B
:10065000D8F4DB01AA59BC4FFD01808191818078DB
:1006600090788030910509F052C0FD01A281B381DC
:10067000A078B078A030B10509F049C0FB013496EC
:1006800061327105BF0128F3E832F10508F444C076
:1006900094C0A52FBB27A85EBD4F6C91643099F024
:1006A000633009F422C0623009F0B6C0E732F105C8
:1006B00008F0B2C0DF01A959BC4F5C91503C0CF06E
:1006C000ABC0319675C0E732F10508F0A5C0DF0177
:1006D000A959BC4F6C91503F09F42CC0543F09F00C
:1006E0002DC060390CF431C097C0E732F10508F035
:1006F00093C0DF01A959BC4F6C91503E09F43DC035
:100700005D3E09F03EC0603A0CF446C085C0FB0176
:10071000E832F10508F051C0DF01AA59BC4F5C91E5
:1007200055230AF446C0DF011196E732F105FD01B9
:1007300098F343C06059603340F06EC0515F53304E
:1007400008F06AC0603C0CF067C0E632F10508F0C2
:1007500063C0DF01A859BC4F5C91503C0CF05CC0F9
:10076000E532F10508F058C0DF01A759BC4F5C9194
:10077000503C0CF051C033961BC0607E603A61F073
:100780004BC0752F715E7C3020F05E7F5E3E09F0BD
:1007900043C0603C0CF040C0E632F10508F03CC0BC
:1007A000DF01A859BC4F5C91503C0CF035C032962B
:1007B0003196E832F10508F433CFA6E6B3E02EE82F
:1007C00033E04C915091C00050725030D9F34093B7
:1007D000C6001196A217B307A1F720E247EF5FE327
:1007E0006BEF78E003C0CB010197F1F723B9F80173
:1007F000D80107C03170EF5FFF4FAF4FBF4F3030B0
:1008000091F3CA010197F1F731E0E33FF105A00749
:10081000B10780F3312DEECFCE0181579F4F60E0BD
:1008200071E00E9434040E94AF478FBF0E943004E1
:100830000E94AF47CE01815F9E4F68E071E00E9449
:1008400034040E94AF4760E801C060E470E0CA0170
:100850000E94070A0E94AF470E9436100E94AF47CD
:100860000E942C040E94AF470E942C040E94AF47B4
:100870004F925F926F927F928F929F92AF92BF92B0
:10088000CF92DF92EF92FF920F931F93CF93DF935C
:10089000CDB7DEB76A970FB6F894DEBF0FBECDBFF7
:1008A0009B01FC01A081B1818C91803009F440C092
:1008B0004D01F90104811581C680D780F601E680DB
:1008C000F7806CE072E044E050E0C801F7015901A4
:1008D0000995982F81E0903009F096C0D4011196C7
:1008E000F501608171819B012470307040E050E01F
:1008F0002030310544075507950109F4812D3D014C
:100900008170803009F023C0690169E273E041E041
:1009100050E0C801F7010995803009F074C0C301A7
:10092000B6010E94E00DF601803009F06CC084C071
:10093000F9018481958126813781F90126813781EA
:1009400060E172E044E050E0F90109955DC02B01DF
:10095000F901A280B38067E273E042E050E0C80191
:10096000F70149010995982F81E0903009F04CC0BA
:100970008F83CE0107968D839E83CB82DC82098391
:100980001A837401F4018485958522853385408519
:10099000518566857785A189B2891089FE013196D6
:1009A000EC87FD87ECE1F1E0EE87FF87188FA98FD8
:1009B000BA8F6E8B7F8B488B598B2A8B3B8B4886EB
:1009C0005986AA86BB868C8B9D8BBE01685F7F4F44
:1009D000C3018B010E94E00D8030A9F4F801DF0112
:1009E0001696349680819181FD0120813181F90133
:1009F000268137816DE173E042E050E0F90109950D
:100A00008030F701C9F081E099276A960FB6F89413
:100A1000DEBF0FBECDBFDF91CF911F910F91FF9031
:100A2000EF90DF90CF90BF90AF909F908F907F908E
:100A30006F905F904F900895DF01169634968081F5
:100A40009181FD0120813181F901268137816AE29E
:100A500073E041E078CF2F923F924F925F927F9266
:100A60008F929F92AF92BF92CF92DF92EF92FF92BE
:100A70000F931F93CF93DF93CDB7DEB7E6970FB6F3
:100A8000F894DEBF0FBECDBF00E010E009A71AA7A3
:100A90002AE030E02FA338A709A31AA32F8F38A389
:100AA00009AB1AAB21E030E02FA738AB4DA75EA70A
:100AB0000BA71CA74DA35EA36BA37CA34D8F5E8FDA
:100AC0000B8F1C8FFE017B96DF015796A98FBA8F83
:100AD000DF015696AD83BE83DF015496A987BA879E
:100AE000DF015296AD87BE87DF015096AF8BB88F7E
:100AF000DF011A96AB83BC83DF011896AB87BC87F6
:100B0000DF011496AF87B88B3296EF83F887FC012C
:100B1000808191818B8B9C8B848195818D8B9E8B29
:100B2000828193810696898B9A8B11C0A7012170CF
:100B3000AD89BE892C93E989FA89208131818B891D
:100B40009C89B601F9010995803009F05CC1A98D35
:100B5000BA8D8C91803009F054C1ED85FE85E0801E
:100B6000F180EF89F88D20803180EB85FC85C08095
:100B7000D180E214F30408F4E7C0EB81FC814080EB
:100B800051804E145F0408F4DFC0B7016219730985
:100B90004601820C931CC982DA82E985FA8540817C
:100BA0005181DA018F859889A80FB91F11977C9020
:100BB0006430710588F46030710509F4C1C0F80132
:100BC000D401AE0FBF1F8C91871509F478C0319600
:100BD000E617F707A8F3B4C0C40101968E7F881505
:100BE000990509F051C0CB0104975C01C801272D7C
:100BF0003327032F070D102F0027022B132BD401AF
:100C0000A80FB91FFD012081318120273127F9016B
:100C1000E150F140209530952E233F232078307805
:100C200020303105B9F4FD0122813381202731279D
:100C3000F901E150F140209530952E233F23207893
:100C400030782030310531F40496950128173907A2
:100C500008F0D5CF6817790708F4EFC000E010E07E
:100C60006817790709F46CC0880E991E681B790B08
:100C7000F801D401AE0FBF1F2C912715F1F031966A
:100C8000E617F707B0F35CC088199909861797072C
:100C900008F0CB01F801D401AE0FBF1F2C9127152E
:100CA00071F03196E817F907B0F3FB0134975F0153
:100CB000E817F90708F09BCFD3CFE80FF91FE20D33
:100CC000F31D31961F01EF89F88D208231822416A1
:100CD000350608F428C042145304C80128F0C101A5
:100CE000841B950B8C0D9D1D42145304E0F0453080
:100CF000510508F0A6C06F8578890E94B447EF8936
:100D0000F88D208031808030910509F46EC0ED852A
:100D1000FE85E080F180EB81FC8140805180EB8595
:100D2000FC85C080D180E214F30470F04601820C8F
:100D3000931CB701621973094E145F0428F02DCF7C
:100D4000EF89F88DE082F182A98DBA8D8C91803087
:100D500009F057C0A98DBA8D81E08C93EF81F88599
:100D600040815181AD81BE812C918B8D9C8D203035
:100D700021F44817590709F444C0481B590BC80E01
:100D8000D91EAD89BE898C91803089F07A01E989BC
:100D9000FA89208131818B899C8964E172E044E089
:100DA00050E0F9010995A701803009F02CC00DAB86
:100DB0001EAB8AE090E08BAB9CAB40305105212DFF
:100DC00009F4B5CE7A01FA01EC0DFD1D3197CE0183
:100DD000C396BF0141E050E00E94B44721E080305B
:100DE000910509F4A3CE212DA1CE8B8D9C8DC980B8
:100DF000DA80C80ED91EA1014B8F5C8F481B590B9E
:100E0000C0CF812D01C081E09927E6960FB6F894F6
:100E1000DEBF0FBECDBFDF91CF911F910F91FF902D
:100E2000EF90DF90CF90BF90AF909F908F907F908A
:100E30005F904F903F902F9008950E94070A0E9464
:100E4000AF4764E070E0CA010E94070A0E94AF4702
:100E50002F923F924F925F926F927F928F929F92CA
:100E6000AF92BF92CF92DF92EF92FF92CF93DF9338
:100E7000CDB7DEB76C970FB6F894DEBF0FBECDBF0F
:100E800079016A015B019C01D9011296F901828105
:100E900091E0803081E009F0C1C0F9018381408197
:100EA0005181FA0190819470903061F4803009F49E
:100EB00073C06FE173E03D014901803009F073C0F8
:100EC00043E072C0A983BA831901803091F44F01C5
:100ED0008481958126813781F9012681378168E1F6
:100EE00073E043E050E0F9010995F401803009F026
:100EF0004EC081E089878481958126813781AE014A
:100F0000475F5F4F4F8358872D833E838B839C833E
:100F100084859585228133814081518162857385E5
:100F2000A085B18586849784618872885088ECE1B9
:100F3000F1E0E88BF98B5A8E6B8E7C8E888E998EC1
:100F4000AA8BBB8B6C8B7D8B4A875B872C873D87FD
:100F50008E8B9F8BCE0103968E879F87B501A6014E
:100F60000E942B05803099F4CE0103966BE173E06B
:100F700042E050E00E942B05803049F4BE01665FDC
:100F80007F4FC701F8010995803009F467C081E0FF
:100F90009101A981BA8141C061E273E03D0149013B
:100FA000803009F48DCF42E050E02F01848195819B
:100FB00026813781F90126813781F9010995803031
:100FC00009F028C0D2011696F2013496E983FA831B
:100FD000808191811D01FD0120813181F9012681EE
:100FE0003781B501A601F9010995803099F4E981AD
:100FF000FA8180819181F10120813181F90126817D
:1010000037816BE173E042E050E0F90109958030EF
:1010100009F41FC081E09401D30191E08C93F901A0
:101020009383C9016C960FB6F894DEBF0FBECDBF97
:10103000DF91CF91FF90EF90DF90CF90BF90AF9076
:101040009F908F907F906F905F904F903F902F90E8
:101050000895C701B201F8010995DDCFFE013A9666
:10106000DF011696349680819181FD0120813181C6
:10107000F901268137816DE173E042E050E0F9012A
:10108000099586CFCF93DF93CDB7DEB724970FB600
:10109000F894DEBF0FBECDBF20E030E02B833C8351
:1010A00029833A83E1E0403851056207730708F06D
:1010B000E12DE170E03019F0498341E079C0F8E0BA
:1010C000E1E040305F076207730708F0E12DE1704F
:1010D000E03091F0242F2F7320682A835295429597
:1010E0004F7045275F70452756954795569547950C
:1010F000406C498342E05CC0E1E0F0E021E0403038
:1011000051056E077F0708F0212D2170FE013196F1
:10111000DF0112963196203009F422C09A01232F64
:1011200022952F70332772956295707F7627607FA6
:101130007627622B732B606E69839A013295229514
:101140002F7023273F7023273695279536952795AF
:101150002F73206820834F7340684C9343E028C06E
:10116000262F269526952770206F29839A01232FF5
:1011700022952F70332772956295707F7627607F56
:101180007627622B732B6F73606860839A013295A8
:1011900022952F7023273F70232736952795369564
:1011A00027952F7320682C934F7340684C8344E03D
:1011B00050E0BE016F5F7F4F0E942B059927249658
:1011C0000FB6F894DEBF0FBECDBFDF91CF9108956B
:1011D000CF93DF93CDB7DEB72E970FB6F894DEBF6F
:1011E0000FBECDBF89839A83FB01828593858D874E
:1011F0009E87808591858B879C878681978189874B
:101200009A87848195818F839887828193818D834A
:101210009E83808191818B839C83CE010196BE0148
:101220006D5F7F4F0E94130A99272E960FB6F89490
:10123000DEBF0FBECDBFDF91CF910895FC0180814D
:1012400091810E942B0599270895CF93DF93CDB705
:10125000DEB724970FB6F894DEBF0FBECDBFFC01FA
:101260008081918120E030E02B833C8329833A8385
:10127000E1E0403851056207730708F0E12DE170A5
:10128000E03019F0498341E079C0F8E0E1E0403016
:101290005F076207730708F0E12DE170E03091F01D
:1012A000242F2F7320682A83529542954F7045272B
:1012B0005F7045275695479556954795406C4983ED
:1012C00042E05CC0E1E0F0E021E0403051056E0713
:1012D0007F0708F0212D2170FE013196DF01129663
:1012E0003196203009F422C09A01232F22952F70C5
:1012F000332772956295707F7627607F7627622B01
:10130000732B606E69839A01329522952F70232783
:101310003F70232736952795369527952F7320689C
:1013200020834F7340684C9343E028C0262F2695B6
:1013300026952770206F29839A01232F22952F70DD
:10134000332772956295707F7627607F7627622BB0
:10135000732B6F73606860839A01329522952F70AA
:1013600023273F70232736952795369527952F738A
:1013700020682C934F7340684C8344E050E0BE01DA
:101380006F5F7F4F0E942B05992724960FB6F89424
:10139000DEBF0FBECDBFDF91CF910895CF93DF9316
:1013A000CDB7DEB72E970FB6F894DEBF0FBECDBF18
:1013B000FC018081918189839A83FB0182859385D9
:1013C0008D879E87808591858B879C878681978175
:1013D00089879A87848195818F8398878281938179
:1013E0008D839E83808191818B839C83CE01019626
:1013F000BE016D5F7F4F0E94130A99272E960FB68C
:10140000F894DEBF0FBECDBFDF91CF9108950E944B
:101410000B0A0E94AF470E942C040E94AF47FC01B8
:1014200080819181FFCF2F923F924F925F926F9276
:101430007F928F929F92AF92BF92CF92DF92EF9264
:10144000FF920F931F93CF93DF93CDB7DEB7A19792
:101450000FB6F894DEBF0FBECDBF20E030E0298F7D
:101460003A8F40E250E04F8B588F298B3A8B2F8771
:10147000388B1F8E23E030E02B8F3C8F20E131E052
:101480002D8B3E8B8B8B9C8B9E01215F3F4FC90127
:1014900006968D879E877901C90104968B879C8764
:1014A000FB018081918180302C0191056B837C83CD
:1014B00009F4F0C04281538181E15802102D1124BA
:1014C000489F212D1124403049835A83510509F446
:1014D0002DC1C701FC017096E987FA87FC013D9692
:1014E000EF83F887FC013C96ED83FE83FC01389680
:1014F0007F01210F322F2227002D1127022B132BC2
:101500009201020F131FFC0171964F010E961C01F0
:10151000FB01C084D184A480B580E0E0F0E03F010D
:10152000CF01880F991F880F991F8A0D9B1DFC0101
:10153000428153814030510599F0FC0160817181F5
:10154000EB85FC8580819181ED85FE85208131814F
:10155000F90126813781F9010995803009F013C11D
:10156000F2018681978120853185BF01A701FA01AB
:101570002283338380839183FB018285AD81BE8189
:101580008C938281938124813581298B3A8B8F873B
:10159000988B2685878590892030B9F02130212DC0
:1015A00009F020C0880F991F880F991F8C0D9D1D71
:1015B000FC01428153816FE07AE04617570739F00A
:1015C00021E04617570769F40DC021E00BC0FC016C
:1015D00080819181FC018081918121E0461757072C
:1015E00009F0212DAF81B8852C93F101808391837F
:1015F000F2012385848595852030B9F02130212D95
:1016000009F020C0880F991F880F991F8C0D9D1D10
:10161000FC01428153816FE07AE04617570739F0A9
:1016200021E04617570769F40DC021E00BC0FC010B
:1016300080819181FC018081918121E046175707CB
:1016400009F0212DA985BA852C93F401808391831B
:10165000F20180819181880F991F880F991F8C0D4D
:101660009D1DFC018081918122813381BE01615FDA
:101670007F4FF9010995803009F085C0F30131965B
:10168000C20141962C018017910709F048CF89814A
:101690009A814EC0028513850030110509F446C0B9
:1016A000FB0180859185000F111F000F111F7C0128
:1016B000080F191FC480D58080E090E09E01215F53
:1016C0003F4F49015C01880F991F880F991F8C0DAE
:1016D0009D1DFC01428153814030510599F0FC0170
:1016E00060817181EB85FC8580819181ED85FE852E
:1016F00020813181F90126813781F90109958030F6
:1017000009F041C0F7018081918122813381B401C8
:10171000F9010995803009F036C0C5010196F7013D
:1017200034967F01E017F10719F0CCCF80E090E00C
:10173000EB81FC81AC01868197819A01481759079A
:1017400008F023C0EB81FC81848195818030910574
:10175000E1F0220F331F220F331F820F931FFC0172
:101760004281538160817181EB85FC85808191810B
:10177000ED85FE8520813181F90126813781F901CE
:101780000995803011F081E001C0812D9927A19643
:101790000FB6F894DEBF0FBECDBFDF91CF911F9182
:1017A0000F91FF90EF90DF90CF90BF90AF909F9000
:1017B0008F907F906F905F904F903F902F90089503
:1017C0002F923F924F925F926F927F928F929F9251
:1017D000AF92BF92CF92DF92EF92FF920F931F933F
:1017E000CF93DF93CDB7DEB72F970FB6F894DEBF58
:1017F0000FBECDBF69017A015B01DC01FD012081D3
:101800003181C9018170907040E050E061E080302A
:1018100091054407550771E009F0712D7170703022
:1018200031F44A875B877030FA0141F009C0E1E189
:10183000F0E0EA87FB877030FA0111F4EBE2F0E0A8
:10184000EC87FD87F901E470F070E030F1054407A2
:10185000550709F0612D6170800F911F603041F0D4
:101860005A01BC01FD018585803009F025C054C0B6
:10187000FD01B70160307105A9F0A501460F571FA2
:1018800060E070E0D50107C07727860E971EB4018F
:10189000A417B50749F04B017D9161E0703CA4F7B6
:1018A000612DF2CF60E070E0680F791FDF01FD016C
:1018B0008585803009F430C0FD01868597853C011F
:1018C0006817790708F028C01B012870307060E0A5
:1018D00070E041E0203031056607770709F0412DBF
:1018E00041704030C886D98609F44EC0FD01948508
:1018F00081E0933009F0892F621873088030AC8240
:10190000BD8209F48EC0813009F091C080E090E082
:101910008A839B83230194C01801FD016680778030
:1019200084809580C401B3012C853D854A855B8503
:1019300085010E94AB0D803011F041E009C0F30138
:1019400026813781C401B601A101F9010995482F0B
:1019500041705070CA012F960FB6F894DEBF0FBECB
:10196000CDBFDF91CF911F910F91FF90EF90DF904E
:10197000CF90BF90AF909F908F907F906F905F902F
:101980004F903F902F9008950E831F83FD01808517
:1019900091858E879F8780E390E0808791878285FD
:1019A00093858A839B83628773878485898381E09B
:1019B000848784809580C680D780C401B6012C8539
:1019C0003D854A855B8585015D010E94AB0D41E047
:1019D000803009F0BDCFF501CF010C968C879D8733
:1019E00038967F01621873085301C60108963C01BE
:1019F00080E090E000E310E01C01DC01C501A817C5
:101A0000B90708F08CC0F301208131811196C4011F
:101A1000A801B101F9012D010995D201803071F3BE
:101A20008CCF80E090E02C016A827B8209C0C301E8
:101A30002C01569447940196969587958A839B83AB
:101A4000FD01828593858E879F87C084D1846480C1
:101A50007580A680B780C50108961C0180E090E0E3
:101A60004C01C20188169906C40170F4F10120816D
:101A7000318101964C01C301A6016E857F85F90174
:101A80000995803071F359CF0E831F8381E190E077
:101A900041E09601203031052E853F852807390722
:101AA00081E009F0812D817080302C853D850C818D
:101AB0001D8109F04DCFC301B5014A855B850E94A8
:101AC000AB0D803009F039CFF50126813781C30194
:101AD000688579854E815F81F9010995803009F02B
:101AE0002CCF80E090E00A811B8141E080179107B4
:101AF00008F0412D8017910708F02ACFF1012081CD
:101B0000318101965C01C3017A01A6016E857F8552
:101B1000F9010995A7018030C50139F319CFF60104
:101B200026813781C401688579854E815F81F901FD
:101B30000995803009F001CFF7018E859F8580835C
:101B400091838A819B81828393838981AC85BD85C2
:101B50008C93412DFDCE8F929F92AF92BF92CF92E8
:101B6000DF92DA015B016C0141E150E081E020305D
:101B70003105A407B50709F0812D8170803061F42B
:101B8000F50180849184C601A901BD01F401099584
:101B9000803011F081E00CC000301105812D41F042
:101BA000F50126813781C601B801A701F901099520
:101BB0009927DF90CF90BF90AF909F908F9008951E
:101BC000EF92FF920F931F93CF93DF93CDB7DEB7C2
:101BD000C058D0400FB6F894DEBF0FBECDBF7B011A
:101BE000DC01F70180819181BC016071707020E09F
:101BF00030E041E0603071052207330709F4412DE0
:101C00004170403009F028C08072907041E080300F
:101C100091052207330709F0412D4170403009F446
:101C200038C01C91812F9927143608F45CC064E6F3
:101C300070E00E949B47880F991FFC01EC5BFE4FF0
:101C4000808191818EA39FA389E2189F112D112479
:101C500012951F7084E24AC04C919E012F5F3F4F46
:101C6000D901A058BF4F80E890E00BC0980F9E9319
:101C7000CF010197542F52955F704031452F08F4E2
:101C800024C0FC01842F8F7090E38A3078F397E5AD
:101C9000EDCF4C919E012F5F3F4FD901A058BF4F10
:101CA00080E890E00AC0980F9E93CF010197542FCF
:101CB00052955F704031452F40F0FC01842F8F70AA
:101CC00090E38A3080F397E3EECF8138910508F0F6
:101CD0003FC0280F391F01E810E00E1B1F0B62E404
:101CE00071E042E022C01A3048F486E290E0DE0162
:101CF0001196A80FB91F105D1C930BC0880F991F78
:101D0000FC01EC5BFE4F808191818EA39FA385E255
:101D100090E09E012F5F3F4F280F391F07E210E030
:101D2000081B190B68E173E040E050E0C7010E9416
:101D3000E00B9927C058DF4F0FB6F894DEBF0FBEF7
:101D4000CDBFDF91CF911F910F91FF90EF9008953C
:101D500060E870E00E94070A0E94AF47AF92BF920E
:101D6000CF92DF92EF92FF920F931F93CF93DF9367
:101D7000CDB7DEB726970FB6F894DEBF0FBECDBF46
:101D80008B017C01F7013296E983FA83F8018481A3
:101D9000958126813781F901268137816BE273E0D5
:101DA00049E050E06A01F90109951E828D830B8399
:101DB0001C83CE01039664E373E04BE050E00AE23B
:101DC0001FE05C0197010E9428076FE373E09E010A
:101DD0002F5F3F4F08E314E0C501A6010E942807CA
:101DE0008D819E81903009F423C0803011F081E014
:101DF0001FC0AB81BC818C918470FD01803059F48F
:101E00008481958126813781F9012681378165E2B8
:101E100073E042E00AC08481958126813781F9010F
:101E20002681378164E273E041E050E0F9010995D1
:101E3000992726960FB6F894DEBF0FBECDBFDF916F
:101E4000CF911F910F91FF90EF90DF90CF90BF90B7
:101E5000AF900895CF92DF92EF92FF920F931F936E
:101E6000CF93DF93CDB7DEB7C058D0400FB6F8940C
:101E7000DEBF0FBECDBF7B01F70120813181F901AB
:101E8000E071F07040E050E061E0E030F1054407BF
:101E9000550709F4612D6170603009F037C0207278
:101EA000307061E0203031054407550709F0612D9D
:101EB0006170FC01603009F44DC00081118187E23E
:101EC0000031180787E290E008F474C06C0160E10B
:101ED00077E2C8010E949B478B0164E670E00E9494
:101EE0009B47880F991FFC01EC5BFE4F808191811D
:101EF0008EA39FA3660F771FFB01EC5BFE4F8081D3
:101F000091818CA39DA383E290E083C0FC0140817A
:101F100051819E012F5F3F4FD901A058BF4F80E8EC
:101F200090E010C0980F9E93CF010197BA0172956F
:101F300062956F7067277F70672740315105AB014D
:101F400008F42AC0FC01842F8F7090E38A3050F38C
:101F500097E5E8CF408151819E012F5F3F4FD90126
:101F6000A058BF4F80E890E00FC0980F9E93CF011C
:101F70000197BA01729562956F7067277F70672726
:101F800040315105AB0140F0FC01842F8F7090E38C
:101F90008A3058F397E3E9CF8138910508F060C0A3
:101FA000280F391F01E810E00E1B1F0B62E471E0DF
:101FB00042E041C004366C01110508F425C064E616
:101FC00070E0C8010E949B478B01880F991FFC019C
:101FD000EC5BFE4F808191818EA39FA385E290E010
:101FE0000A301105B0F002979E012F5F3F4F280F76
:101FF000391F000F111FF801EC5BFE4F408151812A
:10200000F901408351830CC087E290E00A3011054A
:1020100050F70197DE011196A80FB91F005D0C93D0
:1020200086019E012F5F3F4F280F391F081B190B98
:1020300068E173E040E050E0C7010E94E00B99279F
:10204000C058DF4F0FB6F894DEBF0FBECDBFDF9193
:10205000CF911F910F91FF90EF90DF90CF90089557
:1020600060E870E00E94070A0E94AF47FFCFFB01C3
:102070008481958126813781F9012681378168E441
:1020800073E04AE050E0F9010995992708952F92ED
:102090003F924F925F926F927F928F929F92AF92F8
:1020A000BF92CF92DF92EF92FF920F931F93CF9345
:1020B000DF93CDB7DEB7CC59D0400FB6F894DEBF72
:1020C0000FBECDBF7B016C018E01035A1F4F40E450
:1020D00050E0C801612D0E94CA4780E090E09C0159
:1020E000220F331F220F331FF701E20FF31F42812C
:1020F0005381BA01672F7727542F4427462B572B3C
:1021000060817181200F311FF901408351839B0150
:10211000232F3327762F6627622B732B62837383DB
:1021200001968031910509F0DACFF601808491841F
:1021300044845584920128253925E480F5802E2198
:102140003F2124253525828593850FB66D968EAF68
:102150009FAF6D970FBEC684D784860108271927C5
:1021600086819781082319230C251D2540815181E3
:10217000DA015A01B295A295B07FBA27A07FBA279B
:10218000AA0FBB1F42815381E983FA83BA014D83B1
:102190005E83672F77276695669566956A2B7B2BFE
:1021A00052954295507F5427407F5427440F551F26
:1021B000D5013501AB2FBB27A695A695A695A42BD7
:1021C000B52B620F731FA01FB11F008911892289CF
:1021D00033890FB66F96EEADFFAD6F970FBE0FB69A
:1021E0002196EEAFFFAF21970FBE0FB6A1964EAD71
:1021F0005FADA1970FBE4DAF5EAF0E0F1F1F241F27
:10220000351F060F171F2A1F3B1F075616482D475D
:10221000354AA8010FB667960EAF1FAF67970FBE7E
:1022200052954295507F5427407F5427440F551FA5
:10223000D901AB2FBB27A695A695A695A42BB52BA8
:10224000A90152954295507F5427407F5427440F4F
:10225000551F012F1127069506950695042B152B62
:10226000A7015695479556954795FC01FE2FF29587
:10227000F07FEE27FF0FFF0FE42BF52BAF011F01BF
:1022800048255925462157216B827C8248255925AE
:10229000BA019695879596958795A701542F5295E3
:1022A000507F4427550F550F482B592BCA015A010F
:1022B0000FB66D964EAD5FAD6D970FBE8427952717
:1022C000ED80FE808E219F2184279527640D751D4A
:1022D0008C1D9D1D0FB6A396EEADFFADA3970FBE4F
:1022E0000FB62396EEAFFFAF23970FBE0FB6A5969E
:1022F0004EAD5FADA5970FBE49A35AA36E0F7F1FCA
:10230000841F951F6A0F7B1F801F911F6756764899
:102310008D47954AAB010FB669966EAF7FAF69974F
:102320000FBE52954295507F5427407F5427440F4B
:10233000551FFC01EF2FFF27E695E695E695E42B68
:10234000F52BDC01B295A295B07FBA27A07FBA2702
:10235000AA0FBB1FAB01452F5527469546954695BD
:102360004A2B5B2BD301B695A795B695A795B701D8
:10237000762F7295707F6627770F770F6A2B7B2BEE
:102380000FB66B966EAF7FAF6B970FBED101A627CE
:10239000B7270FB667964EAC5FAC67970FBEA42108
:1023A000B521A225B325F694E794F694E79483012A
:1023B000102F1295107F0027110F110F0E291F29C2
:1023C0000FB66596AEAEBFAE65970FBE6501C0266F
:1023D000D126C222D322CA24DB240FB6A796EEACA4
:1023E000FFACA7970FBE0FB62796EEAEFFAE2797AE
:1023F0000FBE0FB6A996AEACBFACA9970FBEABA2ED
:10240000BCA28E0C9F1C0FB66D966EAD7FAD6D9706
:102410000FBE6A1D7B1D8A0E9B1E6C1D7D1DD40187
:10242000AE0FBF1F641F751FA756B6486D47754A8C
:10243000AD017D010FB66396EEAEFFAE63970FBEA2
:1024400052954295507F5427407F5427440F551F83
:10245000DB01FB010FB66D96EEAFFFAF6D970FBEC0
:10246000AB2FBB27A695A695A695A42BB52BF295C9
:10247000E295F07FFE27E07FFE27EE0FFF1FA7010A
:10248000452F55274695469546954E2B5F2BB20115
:102490006B01D694C794D694C794F901FE2FF29598
:1024A000F07FEE27FF0FFF0FEC29FD294F010FB63C
:1024B0006B96EEACFFAC6B970FBE8E249F240FB6CD
:1024C0006996AEACBFAC69970FBE8A209B208E2464
:1024D0009F243695279536952795762F7295707F90
:1024E0006627770F770F622B732B9B013B01202709
:1024F000312728233923202731270FB6AB96CEACBE
:10250000DFACAB970FBE0FB62996CEAEDFAE2997E4
:102510000FBE0FB6AD96EEACFFACAD970FBEE9AAFD
:10252000FAAA2C0C3D1C0FB665966EAD7FAD659773
:102530000FBE6E1D7F1D280C391C621F731F910179
:102540002A0F3B1F641F751F275636486D47754A73
:10255000A90179010FB66596EEAEFFAE65970FBE85
:1025600052954295507F5427407F5427440F551F62
:102570009B012B01232F3327269526952695242B67
:10258000352BD201B295A295B07FBA27A07FBA278A
:10259000AA0FBB1FA701452F55274695469546957F
:1025A0004A2B5B2BD501B695A795B695A795BC018F
:1025B000762F7295707F6627770F770F6A2B7B2BAC
:1025C000DB016B01AE27BF270FB663962EAC3FAC85
:1025D00063970FBEA221B321AE27BF27969587959B
:1025E00096958795B501762F7295707F6627770F40
:1025F000770F682B792BCB014B010FB667966EAE28
:102600007FAE67970FBE862597250FB66D96EEAC09
:10261000FFAC6D970FBE8E219F2186259725A20FB7
:10262000B31F841F951F0FB6AF964EAD5FADAF972A
:102630000FBE0FB62B964EAF5FAF2B970FBE0FB6E8
:10264000E1962EAD3FADE1970FBE2DA33EA30FB691
:102650006B966EAD7FAD6B970FBE640F751F021F3B
:10266000131F6A0F7B1F081F191F675676480D47F7
:10267000154ACB010FB66B966EAF7FAF6B970FBE4F
:1026800092958295907F9827807F9827880F991F31
:10269000A801452F5527469546954695482B592B19
:1026A000980132952295307F3227207F3227220FE2
:1026B000331FCB01892F9927869586958695822B86
:1026C000932BB1019B0136952795369527951701D8
:1026D000D101BA2FB295B07FAA27BB0FBB0FA22B97
:1026E000B32B7D013D01EC24FD240FB66596AEAC05
:1026F000BFAC65970FBEEA20FB20EC24FD249101BE
:102700003695279536952795D9019B01322F32951D
:10271000307F2227330F330F2A2B3B2B1901B101B6
:1027200068257925642175216825792597012E0F63
:102730003F1F0FB66796EEADFFAD67970FBE6E1FDA
:102740007F1F0FB6E396AEADBFADE3970FBEADAB47
:10275000BEAB0FB6E596EEADFFADE5970FBEEF8BC6
:10276000F88F2A0F3B1F6E1F7F1F240F351F681F16
:10277000791F275636486D47754AC9010FB66196CD
:102780002EAF3FAF61970FBE92958295907F9827AD
:10279000807F9827880F991FAB01452F55274695B5
:1027A00046954695482B592BFB01F295E295F07F13
:1027B000FE27E07FFE27EE0FFF1FC901892F992713
:1027C0008695869586958E2B9F2B7501F701F6953C
:1027D000E795F695E7959201322F3295307F2227C3
:1027E000330F330F2E2B3F2B0FB66D962EAF3FAF0F
:1027F0006D970FBEF9010FB669966EAE7FAE699701
:102800000FBEE625F7250FB66B96AEACBFAC6B9747
:102810000FBEEA21FB21E625F725569447945694EE
:102820004794D701BA2FB295B07FAA27BB0FBB0F31
:10283000A429B5290FB66596AEAFBFAF65970FBE99
:102840003D016224732460227122622473240FB636
:10285000E796EEACFFACE7970FBE0FB66796EEAE0D
:10286000FFAE67970FBE0FB6E996AEADBFADE99765
:102870000FBEAFA7B8ABCE0CDF1C8A1E9B1ECE0EC0
:10288000DF1E9401261D371DF601E40FF51F281FDA
:10289000391FE756F6482D47354ACF01DF010FB6FD
:1028A0006396AEAFBFAF63970FBE92958295907F50
:1028B0009827807F9827880F991FA9014901452FE4
:1028C0005527469546954695482B592BF401F29588
:1028D000E295F07FFE27E07FFE27EE0FFF1FCD0180
:1028E000892F99278695869586958E2B9F2BD501C6
:1028F0003D017694679476946794F801FE2FF295E3
:10290000F07FEE27FF0FFF0FE629F7293F010FB6F3
:102910006D962EAD3FAD6D970FBE622673260FB636
:102920006196CEACDFAC61970FBE6C207D20622635
:1029300073261695079516950795BA2FB295B07F11
:10294000AA27BB0FBB0FA02BB12B8D012D010FB6FA
:102950006596AEACBFAC65970FBE0A251B25062356
:1029600017230A251B250FB6EB96EEACFFACEB97B1
:102970000FBEED8EFE8E0FB6ED96AEADBFADED97F0
:102980000FBEAF8FB8A30FB669962EAD3FAD699756
:102990000FBE2E0D3F1D2A1E3B1E260D371D201E6D
:1029A000311E240F351FD101A81FB91F27563648E5
:1029B000AD47B54AC90192958295907F9827807F4F
:1029C0009827880F991FAD017D01452F5527469502
:1029D00046954695482B592B870112950295107FF5
:1029E0001027007F1027000F111FC9013901892FFF
:1029F0009927869586958695802B912BD6018D01FA
:102A000016950795169507959B01322F3295307FC5
:102A10002227330F330F202B312B890119010E2769
:102A20001F270FB66396CEACDFAC63970FBE0C21A9
:102A30001D210E271F277695679576956795BA2FE6
:102A4000B295B07FAA27BB0FBB0FA62BB72B0FB633
:102A50006196AEAFBFAF61970FBE9D010FB66B968B
:102A60004EAE5FAE6B970FBE242535252821392148
:102A700024253525040F151F281F391F0FB6EF9683
:102A80008EAD9FADEF970FBE8BAB9CAB0FB6CF5B00
:102A9000DF4F4EAD5FADC154D0400FBE4FA358A71E
:102AA0000FB66D966EAD7FAD6D970FBE680F791F37
:102AB000D501A41FB51F600F711FA21FB31F67565A
:102AC0007648AD47B54ACB010FB66D966EAF7FAF76
:102AD0006D970FBE92958295907F9827807F98275B
:102AE000880F991F8D015D01012F1127069506950D
:102AF0000695082B192B950132952295307F3227A8
:102B0000207F3227220F331FCB01892F99278695EB
:102B100086958695822B932BD6019D013695279518
:102B200036952795A401542F5295507F4427550F71
:102B3000550F422B532B9A012A012225332563017D
:102B40002C213D2122253325B90196948794969412
:102B500087949D01322F3295307F2227330F330F18
:102B600028293929D90139010FB661968EAC9FAC5D
:102B700061970FBEA825B925AE21BF21A825B9258B
:102B80006E0F7F1F0FB66B962EAD3FAD6B970FBECE
:102B9000A21FB31F0FB6CD5BDF4F4EAD5FADC35469
:102BA000D0400FBE0FB663964EAF5FAF63970FBEB8
:102BB0000FB6CB5BDF4F2EAD3FADC554D0400FBE3F
:102BC000298F3A8F640F751FA21FB31F600F711FEB
:102BD000A81FB91F67567648AD47B54ACB019B0180
:102BE0000FB665962EAF3FAF65970FBE9295829553
:102BF000907F9827807F9827880F991FFD01EF2FDE
:102C0000FF27E695E695E695E82BF92BBD01729531
:102C10006295707F7627607F7627660F771FC901E0
:102C2000892F9927869586958695862B972B8601E1
:102C3000B80176956795769567959701322F32950D
:102C4000307F2227330F330F262B372B0FB66B968F
:102C50002EAF3FAF6B970FBEB901642575250FB638
:102C60006D96CEACDFAC6D970FBE6C217D216425D7
:102C70007525F694E794F694E794102F1295107F3B
:102C80000027110F110F0E291F290FB669960EAFDD
:102C90001FAF69970FBE062517250A211B210625A0
:102CA00017250FB6C95BDF4F4EAD5FADC754D0409F
:102CB0000FBE4B8F5C8F0FB6C75BDF4F2EAD3FADA6
:102CC000C954D0400FBE298B3A8B240E351EA40167
:102CD000421F531F260E371E401F511F91012E0FFA
:102CE0003F1F481F591F275636484D47554AC901AF
:102CF0000FB661962EAF3FAF61970FBE929582954A
:102D0000907F9827807F9827880F991F8A017A01E2
:102D1000012F1127069506950695082B192BB7014B
:102D200072956295707F7627607F7627660F771F92
:102D3000232F3327269526952695262B372BA6015C
:102D4000BA017695679576956795C501982F929506
:102D5000907F8827990F990F862B972BBC011C0118
:102D60000FB66B968EAD9FAD6B970FBE6827792718
:102D70000FB665968EAC9FAC65970FBE6821792122
:102D800068277927B694A794B694A794542F5295A0
:102D9000507F4427550F550F4A295B290FB66D9672
:102DA0004EAF5FAF6D970FBECA010FB669964EADBD
:102DB0005FAD69970FBE842795278A239B238427BD
:102DC00095270FB6C55BDF4F4EAD5FADCB54D040FE
:102DD0000FBE4BA75CA70FB6C35BDF4FEEADFFADD9
:102DE000CD54D0400FBEED8BFE8B440E551E6E1E93
:102DF0007F1E460E571EB301681F791FA201400FA8
:102E0000511F621F731F475656486D47754ACA01C6
:102E10000FB625964EAF5FAF25970FBE9295829560
:102E2000907F9827807F9827880F991F8B016B01CF
:102E3000012F1127069506950695082B192B96014B
:102E400032952295307F3227207F3227220F331F81
:102E5000CA01892F9927869586958695822B932B73
:102E6000B4019B013695279536952795AD01542FD2
:102E70005295507F4427550F550F422B532B9A01E3
:102E80002A010FB62F962EAE3FAE2F970FBE2225EA
:102E900033250FB66196AEACBFAC61970FBE2A2149
:102EA0003B2122253325B695A795B695A795AB016D
:102EB000542F5295507F4427550F550F4A2B5B2BAB
:102EC0004A010FB66D966EAD7FAD6D970FBE46276A
:102ED00057274E215F2146275727200F311F481FB4
:102EE000591F0FB6C15BDF4F6EAD7FADCF54D040E1
:102EF0000FBE69A77AA70FB6CF5ADF4F8EAD9FAD31
:102F0000C155D0400FBE8B879C870FB66B96EEAD38
:102F1000FFAD6B970FBEE60FF71F0FB669966EAD4C
:102F20007FAD69970FBE681F791FE20FF31F641F03
:102F3000751FE756F6486D47754ACF010FB66B9679
:102F4000EEAFFFAF6B970FBE92958295907F98275B
:102F5000807F9827880F991F9B013B01232F3327E0
:102F6000269526952695282B392BC3019295829577
:102F7000907F9827807F9827880F991FBF01672F20
:102F80007727669566956695682B792B8501C8012C
:102F90009695879596958795A701542F5295507FC2
:102FA0004427550F550F482B592BCA015A01842528
:102FB00095250FB62596AEADBFAD25970FBE8A23DA
:102FC0009B2384259525FC01F694E794F694E794D9
:102FD000C801982F9295907F8827990F990F8E2975
:102FE0009F298C011C01082519250C211D2108256C
:102FF000192574010FB62F968EAD9FAD2F970FBE7A
:10300000E80FF91F0FB66D968EAD9FAD6D970FBE91
:10301000081F191F0FB6CD5ADF4F4EAD5FADC35518
:10302000D0400FBE0FB661964EAF5FAF61970FBE37
:103030000FB6CB5ADF4F8EAD9FADC555D0400FBEFA
:103040008B8B9C8BE40FF51F081F191FE20FF31FDA
:10305000061F171FE756F6480D47154AAF01BF0177
:103060000FB62D966EAF7FAF2D970FBE529542953E
:10307000507F5427407F5427440F551F9801232F1A
:103080003327269526952695242B352BA801529576
:103090004295507F5427407F5427440F551F672F78
:1030A0007727669566956695642B752BFD01AF01B4
:1030B0005695479556954795C601982F9295907FBE
:1030C0008827990F990F842B952B0FB66D968EAF8D
:1030D0009FAF6D970FBEAC014A255B250FB66B966F
:1030E0008EAC9FAC6B970FBE482159214A255B25BA
:1030F000D694C794D694C794CF01982F9295907F79
:103100008827990F990F8C299D29FC016C01E225D4
:10311000F325E621F721E225F3250FB6C95ADF4F43
:10312000AEADBFADC755D0400FBE0FB62F96AEAFF8
:10313000BFAF2F970FBE0FB6C75ADF4F8EAD9FADF3
:10314000C955D0400FBE8F87988B4A0E5B1ED701A2
:10315000A81FB91F440E551EAE1FBF1FC201820F0C
:10316000931FA61FB71F87569648AD47B54A9C01C7
:10317000BC0169AF7AAF32952295307F3227207F2C
:103180003227220F331FFD017D01EF2FFF27E69528
:10319000E695E695E22BF32B970132952295307F49
:1031A0003227207F3227220F331F672F772766951C
:1031B00066956695622B732BC401AC0156954795B5
:1031C000569547959301322F3295307F2227330F42
:1031D000330F242B352BA90129010FB66D962EAD87
:1031E0003FAD6D970FBE422753270FB62D968EAC7D
:1031F0009FAC2D970FBE4821592142275327769423
:10320000679476946794982F9295907F8827990F6A
:10321000990F86299729DC013C010FB62596CEAE81
:10322000DFAE25970FBEAC25BD25A023B123AC256D
:10323000BD250FB6C55ADF4F8EAD9FADCB55D040E3
:103240000FBE8BAF9CAF0FB6C35ADF4F2EAD3FAD55
:10325000CD55D0400FBE2D873E87A80EB91E221E29
:10326000331EA40EB51E91012A1F3B1FC5018E0FF0
:103270009F1F261F371F875696482D47354A6901DD
:10328000AC01BC010FB665966EAF7FAF65970FBE00
:1032900052954295507F5427407F5427440F551F25
:1032A000D601AB2FBB27A695A695A695A42BB52B2B
:1032B000A60152954295507F5427407F5427440FD2
:1032C000551F672F7727669566956695642B752B36
:1032D0009401A9015695479556954795C801982F91
:1032E0009295907F8827990F990F842B952BFC013D
:1032F0004C010FB669964EAE5FAE69970FBEE425DE
:10330000F525A9ACBAACEA21FB21E425F5251695F3
:10331000079516950795322F3295307F2227330F68
:10332000330F202B312BC9011901862597258E21BA
:103330009F2186259725EA0FFB1F861F971F0FB633
:1033400021966EAD7FAD21970FBE0FB627962EAD9D
:103350003FAD27970FBE622773272BA93CA9622791
:1033600073270FB661962EAD3FAD61970FBE6227F2
:103370007327AB01440F551F2DAD3EADABA1BCA1D2
:103380002A273B27AFA1B8A52A273B27AB89BC89B1
:103390002A273B27D901AB2FA295AF70BB27A69553
:1033A000A695A695A42BB52BADAFBEAF220F331FAC
:1033B000672F62956F707727669566956695622B85
:1033C000732B0FB621966EAF7FAF21970FBE0FB64E
:1033D0006D962EAD3FAD6D970FBE2A0F3B1F0FB6FA
:1033E00025960EAD1FAD25970FBE061F171F2E0F7A
:1033F0003F1F081F191F275636480D47154AC90198
:103400000FB66D962EAF3FAF6D970FBE929582951A
:10341000907F9827807F9827880F991FF801EF2FBA
:10342000FF27E695E695E695E82BF92BA80152953E
:103430004295507F5427407F5427440F551FC901A0
:10344000892F9927869586958695842B952BA5019E
:1034500056954795569547959701322F3295307F6F
:103460002227330F330F242B352B2DA73EA7A9017D
:1034700094012FAB38AF422753270FB665968EAC19
:103480009FAC65970FBE4821592142275327F694D8
:10349000E794F694E7949501322F3295307F2227F6
:1034A000330F330F2E293F29B901290162257325D6
:1034B0006C217D21622573250FB669962EAD3FAD37
:1034C00069970FBE420F531F661D771D5B010FB634
:1034D00023966EAD7FAD23970FBE0FB629962EAD06
:1034E0003FAD29970FBE622773270FB663962EADA7
:1034F0003FAD63970FBE622773270FB62F962EAD91
:103500003FAD2F970FBE622773279B01220F331FFA
:10351000E9A0FAA0A9A9BAA9EA26FB26A98DBA8D25
:10352000EA26FB26AF85B889EA26FB26D701AB2F12
:10353000A295AF70BB27A695A695A695A22BB32BF7
:10354000A9A3BAA3EE0CFF1C672F62956F707727B3
:103550006695669566956E297F290FB623966EAFA0
:103560007FAF23970FBE4A0F5B1F9501261F371FA2
:103570004E0F5F1F281F391F475656482D47354AA3
:10358000CA01DA010FB66B96AEAFBFAF6B970FBE35
:1035900092958295907F9827807F9827880F991F12
:1035A000A9013901452F5527469546954695482B43
:1035B000592BB30172956295707F7627607F7627CD
:1035C000660F771FAB2FBB27A695A695A695A62BB2
:1035D000B72B9401B9017695679576956795C601E5
:1035E000982F9295907F8827990F990F862B972B6C
:1035F0000FB669968EAF9FAF69970FBEBC018DA5C0
:103600009EA5682779270FB66D968EAC9FAC6D97F7
:103610000FBE6821792168277927D694C794D6945C
:10362000C794C901982F9295907F8827990F990F79
:103630008C299D29FC016C0149AE5AAEE425F52583
:10364000E023F123E425F5250FB627964EAC5FACB9
:1036500027970FBE0FB62B968EAD9FAD2B970FBE43
:10366000482659268B8D9C8D482659268BAD9CADBE
:10367000482659265201AA0CBB1C8DA19EA1EBA085
:10368000FCA0E826F92689899A89E826F9268D85FD
:103690009E85E826F926C701892F82958F70992784
:1036A0008695869586958A299B295C010FB6259675
:1036B000AEAEBFAE25970FBEEE0CFF1CC201892F28
:1036C00082958F7099278695869586958E299F2954
:1036D0000FB627968EAF9FAF27970FBEEFA8F8AC17
:1036E000EA0CFB1C9101281F391FC701860F971F89
:1036F0002E1F3F1F840F951F2A1F3B1F875696487A
:10370000AC012D47354AFA01EFABF8AF929582959F
:10371000907F9827807F9827880F991FA9010FB65F
:103720002D962EAF3FAF2D970FBE452F55274695AF
:1037300046954695482B592B32952295307F322756
:10374000207F3227220F331FCF01892F992786959B
:1037500086958695822B932B9401F901F695E79532
:10376000F695E795B801762F7295707F6627770FEB
:10377000770F6E2B7F2BFB010FB66996AEADBFADF9
:1037800069970FBEEA27FB270FB66B962EAC3FACAE
:103790006B970FBEE221F321EA27FB2716950795C9
:1037A00016950795322F3295307F2227330F330F2E
:1037B000202B312B0FB66D962EAF3FAF6D970FBEFE
:1037C00079010FB66596CEAEDFAE65970FBEEC24DD
:1037D000FD24E620F720EC24FD240FB629964EACFC
:1037E0005FAC29970FBEADA9BEA94A265B26ABA543
:1037F000BCA54A265B26ADADBEAD4A265B2652016E
:10380000AA0CBB1C89A89AA8AF89B88D8A269B26CA
:10381000AD89BE898A269B260FB621962EAD3FAD77
:1038200021970FBE82269326D401AB2FA295AF70AD
:10383000BB27A695A695A695AA29BB29A9ABBAAB85
:10384000880C991C9201232F22952F7033272695DF
:1038500026952695282939290FB629962EAF3FAFF0
:1038600029970FBECDA4DEA4CA0EDB1E09AD1AAD8A
:10387000021F131FD601AE0FBF1F0E1D1F1DA40F69
:10388000B51F081F191FA756B6480D47154ACD0189
:1038900092958295907F9827807F9827880F991F0F
:1038A00098016801232F3327269526952695282BE6
:1038B000392BC60192958295907F9827807F982713
:1038C000880F991FFD012D01EF2FFF27E695E69543
:1038D000E695E82BF92BA101CA0196958795969557
:1038E0008795D301BA2FB295B07FAA27BB0FBB0F24
:1038F000A82BB92BCD014D018BA29CA2862797271F
:103900002FA838AC82259325769467947694679493
:10391000542F5295507F4427550F550F462957294C
:103920000FB66B964EAF5FAF6B970FBE0FB66D962F
:10393000AEADBFAD6D970FBE4A275B270FB62D9674
:10394000EEACFFAC2D970FBE4E255F25820F931F67
:103950004E1F5F1F0FB62B96EEADFFAD2B970FBE20
:103960000FB667962EAD3FAD67970FBEE227F327E0
:1039700029A53AA5E227F32729A13AA1E227F327AF
:103980009F01220F331F0DA11EA1AFA5B8A90A27C1
:103990001B27AB85BC850A271B270FB62396AEAD28
:1039A000BFAD23970FBE0A271B27D801AB2FA295C7
:1039B000AF70BB27A695A695A695A22BB32BADA35A
:1039C000BEA3000F111FEF2FE295EF70FF27E695C2
:1039D000E695E695E02BF12B0FB62B96EEAFFFAFF9
:1039E0002B970FBE0FB669960EAD1FAD69970FBE30
:1039F0000A0F1B1F0FB665962EAD3FAD65970FBE24
:103A00002E1F3F1F080F191F241F351F0F5514416C
:103A100026423149C8010FB669960EAF1FAF6997AC
:103A20000FBE92958295907F9827807F9827880F68
:103A3000991FF9015901EF2FFF27E695E695E695C5
:103A4000E82BF92B32952295307F3227207F3227C1
:103A5000220F331FC801892F992786958695869551
:103A6000822B932BD1019D0136952795369527956D
:103A70008701A801542F5295507F4427550F550FA9
:103A8000422B532B7A013A010FB665966EAE7FAE8C
:103A900065970FBEE824F9244201E824F92498012F
:103AA0003695279536952795A9019D01322F329598
:103AB000307F2227330F330F242B352B29014FAAB8
:103AC00058AE0FB66B964EAD5FAD6B970FBE242709
:103AD00035272C253D25E60EF71E0FB66D964EAD0B
:103AE0005FAD6D970FBE241F351F0DA91EA94D8D0B
:103AF0005E8D042715270FB661964EAD5FAD6197B9
:103B00000FBE042715270FB625964EAD5FAD25973E
:103B10000FBE04271527B801660F771F4F89588DF0
:103B2000AF8DB8A14A275B27AB89BC894A275B27A1
:103B30000FB62796AEADBFAD27970FBE4A275B27BE
:103B4000DA01AB2FA295AF70BB27A695A695A695D7
:103B5000A62BB72B0FB62D96AEAFBFAF2D970FBECE
:103B6000440F551F012F02950F70112706950695DA
:103B70000695042B152B0DAB1EABA7014A0F5B1F3F
:103B8000201F311F4E0F5F1F281F391F4F555441F3
:103B900026423149CA0149875A8792958295907F7A
:103BA0009827807F9827880F991FB901672F77275B
:103BB000669566956695682B792BF901F295E295E5
:103BC000F07FFE27E07FFE27EE0FFF1FCA01892F3F
:103BD00099278695869586958E2B9F2BD401FD017E
:103BE000F695E795F695E795A601542F5295507FE7
:103BF0004427550F550F4E2B5F2BFA014A0189AE12
:103C00009AAEE625F7250FB669966EAC7FAC69973C
:103C10000FBEE625F725D694C794D694C794AD0178
:103C2000542F5295507F4427550F550F4C295D292D
:103C30008A011A012DA63EA6042515250A251B2555
:103C40000FB66796CEACDFAC67970FBE4BA95CA9E9
:103C5000C426D5260FB62F964EAD5FAD2F970FBE5B
:103C6000C426D52649A95AA9C426D5267601D60147
:103C7000EE0CFF1CCFA4D8A84FA158A5C426D5266A
:103C80004F855889C426D5260FB629964EAD5FAD0F
:103C900029970FBEC426D526A601452F42954F7001
:103CA00055274695469546954E295F294FA758AB0F
:103CB000CC0CDD1CAB2FA295AF70BB27A695A695AB
:103CC000A695AC29BD290FB66796AEAFBFAF679773
:103CD0000FBEEBA0FCA0E40EF51E0FB66B96CEACAB
:103CE000DFAC6B970FBECA1EDB1EA7014E0F5F1F16
:103CF000F601E01FF11F460F571FE81FF91F4F5530
:103D00005441E642F149CA014BA35CA392958295C6
:103D1000907F9827807F9827880F991FBF012F01D8
:103D2000672F7727669566956695682B792BF295B0
:103D3000E295F07FFE27E07FFE27EE0FFF1FCA010E
:103D4000892F99278695869586958E2B9F2BA30183
:103D50008A011695079516950795F501FE2FF295A0
:103D6000F07FEE27FF0FFF0FE02BF12B8F010825CF
:103D7000192569847A8406251725B694A794B694E4
:103D8000A794542F5295507F4427550F550F4A2919
:103D90005B290FB669964EAF5FAF69970FBE7A0188
:103DA000E224F324E226F326AD8CBE8C0FB6639694
:103DB0004EAD5FAD63970FBEA426B5264BAD5CAD8F
:103DC000A426B5264DA15EA1A426B5266501CC0C7E
:103DD000DD1C4F8D58A1A98DBA8D4A275B27AD8573
:103DE000BE854A275B270FB62B96AEADBFAD2B978E
:103DF0000FBE4A275B27DA014A01AB2FA295AF70AD
:103E0000BB27A695A695A695AC29BD29AD010FB6F1
:103E10006B964EAF5FAF6B970FBE880C991CD501A8
:103E2000AB2FA295AF70BB27A695A695A695A829FE
:103E3000B929AD8FBE8F0FB66596CEACDFAC659756
:103E40000FBEC40ED51EAFA8B8ACAA1EBB1EA601DD
:103E5000400F511FD501AE1DBF1D460F571FA81F94
:103E6000B91F4F555441A642B149CA010FB66596D4
:103E70004EAF5FAF65970FBE92958295907F982762
:103E8000807F9827880F991FBD011D01672F772715
:103E9000669566956695682B792B8101129502953A
:103EA000107F1027007F1027000F111FCA01892FD4
:103EB0009927869586958695802B912B7301F6948C
:103EC000E794F694E794A901542F5295507F442724
:103ED000550F550F4E295F297A015A01AF8EB8A2AE
:103EE000EE26FF26CBA0DCA0EC24FD2436952795FA
:103EF00036952795A301542F5295507F4427550F8F
:103F0000550F422B532B9A014A0189869A860FB688
:103F100069964EAD5FAD69970FBE242735272425DE
:103F20003525E60EF71E281F391F6BA97CA98B8D3E
:103F30009C8D682779278DAD9EAD682779270FB6B0
:103F40002D968EAD9FAD2D970FBE68277927CB019B
:103F5000880F991F4FA158A5A989BA894A275B27BD
:103F60000FB62196AEADBFAD21970FBE4A275B2796
:103F7000ADA9BEA94A275B27DA01AB2FA295AF7086
:103F8000BB27A695A695A695A82BB92BAFA3B8A736
:103F9000440F551F672F62956F707727669566955A
:103FA0006695642B752B6BAB7CAB09AD1AAD0A0F14
:103FB0001B1F4DA55EA5461F571F0E0D1F1D421F3F
:103FC000531F0F55144146425149C80109AF1AAF5A
:103FD00092958295907F9827807F9827880F991FC8
:103FE000BA013A01672F7727669566956695682B23
:103FF000792B930132952295307F3227207F32270B
:10400000220F331FC801892F99278695869586959B
:10401000822B932BD6019D013695279536952795B2
:10402000A201542F5295507F4427550F550F422B14
:10403000532B7A016A01CF8AD88EEA24FB240FB66B
:1040400065964EAD5FAD65970FBEE426F526569496
:104050004794569447949D01322F3295307F222702
:10406000330F330F24293529D9015901ABA2BCA242
:10407000A825B925A225B325EE0EFF1E0FB6699619
:104080002EAD3FAD69970FBEA21FB31F0FB663964B
:104090002EAD3FAD63970FBEEBA5FCA52E273F27A6
:1040A000E9A1FAA12E273F27EFA5F8A92E273F2740
:1040B000F9012901EE0FFF1F2D893E89098D1A8D07
:1040C000022713270FB623962EAD3FAD23970FBEC1
:1040D000022713270FB667962EAD3FAD67970FBE29
:1040E000022713279801232F22952F703327269517
:1040F000269526952E2B3F2BF901EDA7FEA7000F45
:10410000111F9201232F22952F7033272695269574
:104110002695202B312B0FB663962EAF3FAF6397BA
:104120000FBE87010E0F1F1FA21FB31F060F171F01
:10413000A81FB91F0F551441A642B149C8010F83EA
:10414000188792958295907F9827807F9827880F6F
:10415000991FBD01672F7727669566956695682B31
:10416000792BFD01F295E295F07FFE27E07FFE2797
:10417000EE0FFF1FC801892F992786958695869592
:104180008E2B9F2B8A01F801F695E795F695E7951A
:104190009101322F3295307F2227330F330F2E2B90
:1041A0003F2B298F3A8FF901EC25FD2549AD5AADFA
:1041B000E427F52736942794369427949801322FD4
:1041C0003295307F2227330F330F222933290FB640
:1041D00065962EAF3FAF65970FBE7901EA24FB24A9
:1041E000E624F7242B8D3C8D09A51AA5202731271D
:1041F0000FB625960EAD1FAD25970FBE2027312790
:104200000FB66B960EAD1FAD6B970FBE20273127F3
:1042100069012901CC0CDD1C89889A882B853C8595
:10422000822693260FB627962EAD3FAD27970FBE59
:10423000822693262D8D3E8D822693269401232F50
:1042400022952F7033272695269526952C293D29D2
:1042500089010FB66D960EAF1FAF6D970FBE880C1C
:10426000991C9201232F22952F703327269526958E
:104270002695282939292B8F3C8FCF8CD8A0C00EAA
:10428000D11E09851A85021F131F96012E0F3F1F8D
:104290000E1D1F1D260F371F081F191F2F553441D4
:1042A00006421149C9012F8F38A392958295907FBC
:1042B0009827807F9827880F991FF8012801EF2FF2
:1042C000FF27E695E695E695E82BF92BB201729566
:1042D0006295707F7627607F7627660F771FC9010A
:1042E000892F9927869586958695862B972B9A01F7
:1042F0007901F694E794F694E794B301762F7295DA
:10430000707F6627770F770F6E297F297B01498D94
:104310005A8DE426F5262F803884E224F3247694FF
:10432000679476946794322F3295307F2227330F2B
:10433000330F2629372929AF3AAF69010FB66596A1
:104340002EAD3FAD65970FBEC226D326CA26DB260B
:104350002BA53CA50FB661964EAD5FAD61970FBE24
:104360002427352749A95AA9242735274FA158A51D
:10437000242735275901A901AA0CBB1C0D891E89C8
:104380002B893C89022713270FB629962EAD3FAD06
:1043900029970FBE022713272BA93CA90227132711
:1043A00098014801232F22952F70332726952695B3
:1043B00026952A293B2989010FB669960EAF1FAFB2
:1043C00069970FBE880C991C9A01232F22952F7094
:1043D0003327269526952695282939292BA73CA7EA
:1043E0004F89588D400F511F0BA11CA1021F131F95
:1043F0004E0D5F1D0C1D1D1D4E0F5F1F081F191F49
:104400004F55544106421149CA014F8B588F92951E
:104410008295907F9827807F9827880F991FF801B1
:10442000EF2FFF27E695E695E695E82BF92B980107
:1044300032952295307F3227207F3227220F331F7B
:10444000CA01892F9927869586958695822B932B6D
:10445000610196013695279536952795AD01542F24
:104460005295507F4427550F550F422B532B7A01FD
:104470001A01298A3A8AE626F7268F8C98A0E82422
:10448000F924B695A795B695A7959601322F329542
:10449000307F2227330F330F2A2B3B2BD9013901D1
:1044A0006F82788629AD3AADA227B327A425B5251A
:1044B000EE0EFF1EA81FB91F29A53AA50FB62F960D
:1044C0008EAD9FAD2F970FBE282739278DA19EA1B6
:1044D000282739278DA59EA528273927C9015901E5
:1044E000880F991FEB85FC852F853889E227F327F4
:1044F0000FB62B962EAD3FAD2B970FBEE227F327BD
:104500000FB663962EAD3FAD63970FBEE227F3273C
:104510009F01232F22952F703327269526952695C8
:10452000282B392B2BA33CA3EE0FFF1FC501892F8E
:1045300082958F7099278695869586958E2B9F2BD1
:1045400089A79AA7E98DFA8DE20FF31F0FB665963A
:104550004EAD5FAD65970FBE481F591FEE0DFF1D95
:104560004A1F5B1FEF55F441464251499F01DF014D
:10457000A98FBA8F32952295307F3227207F32273C
:10458000220F331FFA015A01EF2FFF27E695E69518
:10459000E695E22BF32B950132952295307F322759
:1045A000207F3227220F331FAB2FBB27A695A6955E
:1045B000A695A22BB32B9401369527953695279572
:1045C000A201542F5295507F4427550F550F422B6F
:1045D000532BCA016A01CD8ADE8A822593252F8852
:1045E000388C822593255694479456944794940189
:1045F000322F3295307F2227330F330F242935296C
:10460000290149018F8E98A246245724402651261D
:10461000860F971F29AD3AAD421E531E0FB6619605
:104620006EAD7FAD61970FBE2BAD3CAD622773279A
:104630000FB62D962EAD3FAD2D970FBE6227732777
:104640000FB66D962EAD3FAD6D970FBE62277327E7
:104650009B01220F331FEB88FC884D855E85E42685
:10466000F5264DA95EA9E426F5264B8D5C8DE42642
:10467000F526A701452F42954F705527469546953B
:104680004695422B532B4FAB58AFEE0CFF1C672FB8
:1046900062956F7077276695669566956E297F2976
:1046A0000FB661966EAF7FAF61970FBE840F951FF7
:1046B000A201461F571F8E0F9F1F4A1F5B1F8F555A
:1046C0009441464251499C01BC016B877C873295DD
:1046D0002295307F3227207F3227220F331FCA01D5
:1046E000FA01892F9927869586958695822B932B9B
:1046F0009F0132952295307F3227207F3227220F6B
:10470000331F672F7727669566956695622B732B07
:10471000710197013695279536952795A801542F55
:104720005295507F4427550F550F422B532BDA01DA
:104730001A012B8A3C8AAC25BD25498C5A8CA425AC
:10474000B52516950795169507959701322F329541
:10475000307F2227330F330F202B312B2F8B388FB5
:104760007901E824F924EA24FB240FB62F962EAD14
:104770003FAD2F970FBE4DAD5EAD242735274FA51A
:1047800058A9242735270FB669964EAD5FAD6997B6
:104790000FBE24273527A901220F331FCF84D888C5
:1047A0000FB621960EAD1FAD21970FBEC026D126A4
:1047B0000FB667966EAC7FAC67970FBEC624D72442
:1047C0000BA51CA5C026D1268601012F02950F70CE
:1047D0001127069506950695022B132B0FB66596A5
:1047E0000EAF1FAF65970FBECC0CDD1C452F429559
:1047F0004F7055274695469546954C295D290FB62D
:104800002F964EAF5FAF2F970FBE29893A89200FA1
:10481000311F0F811885041F151FA9014A0F5B1F47
:104820000E1D1F1D480F591F061F171F4F555441BE
:10483000064211499A01DA01A98BBA8B3295229569
:10484000307F3227207F3227220F331FC8014801D3
:10485000892F9927869586958695822B932B94018F
:1048600032952295307F3227207F3227220F331F47
:10487000AB2FBB27A695A695A695A22BB32BB2016D
:104880009B013695279536952795A501542F52956E
:10489000507F4427550F550F422B532B7A013A0175
:1048A00069867A86E224F3244B845C84E424F5242C
:1048B000B694A794B694A7949B01322F3295307F7B
:1048C0002227330F330F2A293B2969015901A98E69
:1048D000BA8E2F89388DC226D326CE26DF262BAD61
:1048E0003CAD49A15AA1242735270FB66B964EAD92
:1048F0005FAD6B970FBE242735274BA15CA1242702
:104900003527A901220F331F0D851E850FB623966B
:104910006EAD7FAD23970FBE062717276D8D7E8D59
:104920000627172769A57AA506271727B801672F35
:1049300062956F707727669566956695622B732BE7
:1049400069AF7AAF000F111F452F42954F70552761
:10495000469546954695402B512B4BAF5CAF2D8924
:104960003E89260F371F6F8D78A1641F751F2E0D8E
:104970003F1D6C1D7D1D280F391F6A1F7B1F2F5582
:10498000344166427149C901A9014D8B5E8B9295F4
:104990008295907F9827807F9827880F991FDB0149
:1049A0006B01AB2FBB27A695A695A695A82BB92B77
:1049B000960132952295307F3227207F3227220FB1
:1049C000331FCA01892F9927869586958695822B54
:1049D000932BB2019B013695279536952795AF010C
:1049E000542F5295507F4427550F550F422B532B70
:1049F0007A018A010F87188BE624F72469887A8860
:104A0000E624F724F695E795F695E7959B01322F76
:104A10003295307F2227330F330F2E2B3F2BA901E6
:104A200019012B863C864A255B2548255925EA0E27
:104A3000FB1E481F591F2DAD3EAD0FB625968EADFE
:104A40009FAD25970FBE282739278FA198A5282726
:104A500039278FA998AD28273927C901B901880FAF
:104A6000991F0FB62196AEADBFAD21970FBE0FB601
:104A700027962EAD3FAD27970FBEA227B3272BA9B0
:104A80003CA9A227B3270FB661962EAD3FAD619723
:104A90000FBEA227B3279D01232F22952F70332706
:104AA000269526952695282B392B2F8F38A3AA0FCC
:104AB000BB1FCB01892F82958F709927869586958C
:104AC00086958A2B9B2B8DAF9EAF6B897C89620F5D
:104AD000731FEF89F88DE81FF91F6E0D7F1DE41F0E
:104AE000F51F6F557441E642F1499B01DB01AB8B29
:104AF000BC8B32952295307F3227207F3227220FC0
:104B0000331FCF015F01892F99278695869586955A
:104B1000822B932B950132952295307F3227207F6F
:104B20003227220F331FAB2FBB27A695A695A6953C
:104B3000A22BB32BB3019B0136952795369527956C
:104B4000A401542F5295507F4427550F550F422BE7
:104B5000532B7A012A014F8A588EE026F1266D8860
:104B60007E88E624F72496948794969487949B01F4
:104B7000322F3295307F2227330F330F28293929DE
:104B8000A9014901898A9A8A422553254C255D2528
:104B900029853A85E20EF31E298D3A8D421F531F57
:104BA00029A13AA169A97AA9262737276DA57EA54B
:104BB000262737270FB665966EAD7FAD65970FBE7A
:104BC00026273727B901F901660F771F0FB62396FD
:104BD0000EAD1FAD23970FBE0FB629962EAD3FAD7C
:104BE00029970FBE022713270FB663962EAD3FAD50
:104BF00063970FBE022713270FB62F962EAD3FAD3A
:104C00002F970FBE022713279801232F22952F706D
:104C10003327269526952695262B372BB9010FB6D7
:104C200021966EAF7FAF21970FBE000F111F9F011E
:104C3000232F22952F703327269526952695202BF6
:104C4000312B29A33AA3F701E60FF71F421F531F89
:104C5000E80FF91F4A1F5B1FEF55F44146425149C7
:104C60009F011F0132952295307F3227207F322706
:104C7000220F331FCA01892F99278695869586951D
:104C8000822B932B9A0132952295307F3227207FF9
:104C90003227220F331FB101672F7727669566955C
:104CA0006695622B732B930136952795369527953C
:104CB000D601BA2FB295B07FAA27BB0FBB0FA22B8C
:104CC000B32BA98FBA8FA425B5254B885C88A42562
:104CD000B525D694C794D694C7948301102F129506
:104CE000107F0027110F110F0C291D290D8B1E8B12
:104CF000082519250A251B250FB625962EAD3FAD93
:104D000025970FBEEDA1FEA12E273F270FB66D966A
:104D1000EEADFFAD6D970FBE2E273F27E9ADFAAD83
:104D20002E273F277901220F331F0FB627966EAC2F
:104D30007FAC27970FBE0FB62B96EEADFFAD2B972E
:104D40000FBE6E267F26EB8DFC8D6E267F26EBAD8B
:104D5000FCAD6E267F26F301EF2FE295EF70FF2763
:104D6000E695E695E695E22BF32B0FB62396EEAF8C
:104D7000FFAF23970FBE660C771C9701232F229558
:104D80002F703327269526952695262937290FB685
:104D900025962EAF3FAF25970FBEEF84F888EE0E15
:104DA000FF1EEB85FC85E21FF31F97012A0F3B1FB7
:104DB000E01FF11F280F391FE61FF71F2F55344141
:104DC000E642F149C901D901AF87B88B9295829526
:104DD000907F9827807F9827880F991FBF014F01E8
:104DE000672F7727669566956695682B792BC401A2
:104DF00092958295907F9827807F9827880F991F9A
:104E0000AB2FBB27A695A695A695A82BB92BF2018B
:104E10009F013695279536952795C501982F929530
:104E2000907F8827990F990F822B932B8C013C013F
:104E30006B867C86898D9A8D082719270225132574
:104E4000B694A794B694A794CF01982F9295907F8B
:104E50008827990F990F8A299B297C016C01CB8A9D
:104E6000DC8A8D899E89E826F926E426F52629A97B
:104E70003AA90FB62D968EAD9FAD2D970FBE282760
:104E800039270FB669968EAD9FAD69970FBE28275B
:104E900039278F8D98A128273927C901220F331F61
:104EA0000FB62996AEACBFAC29970FBEEDA9FEA9EF
:104EB000AE26BF26EBA5FCA5AE26BF26EDADFEAD0A
:104EC000AE26BF26F501EF2FE295EF70FF27E6959E
:104ED000E695E695E22BF32B0FB62796EEAFFFAFE4
:104EE00027970FBEAA0CBB1C892F82958F7099271C
:104EF0008695869586958A299B2989AB9AAB2F89B9
:104F0000388D2E0F3F1FE989FA89E81FF91FC90163
:104F1000800F911FEE1DFF1D860F971FEA1FFB1FBD
:104F20008F559441E642F1499C018C010F8B188FFB
:104F300032952295307F3227207F3227220F331F70
:104F4000DF017F01AB2FBB27A695A695A695A22BC7
:104F5000B32B970132952295307F3227207F32275D
:104F6000220F331F012F1127069506950695022B58
:104F7000132B91013695279536952795CA01982FC1
:104F80009295907F8827990F990F822B932BBC01C4
:104F90002C014D865E8666257725AF84B8886A2504
:104FA0007B255695479556954795C101982F929523
:104FB000907F8827990F990F842B952B9C011C01BA
:104FC00029863A862C253D25282539256A0F7B1F01
:104FD000201F311F8DA19EA14FA558A98427952779
:104FE0004BA15CA1842795270FB621964EAD5FADEE
:104FF00021970FBE84279527AC01440F551F0FB68C
:105000002B960EAD1FAD2B970FBE0FB66796EEAD6C
:10501000FFAD67970FBE0E271F27E9A5FAA50E273C
:105020001F27E9A1FAA10E271F27D801AB2FA295B0
:10503000AF70BB27A695A695A695A42BB52B0FB64A
:105040002996AEAFBFAF29970FBE000F111FAC015D
:10505000452F42954F705527469546954695402BCE
:10506000512B4DA35EA3898D9A8D8A0F9B1FED89CD
:10507000FE89E41FF51F860F971FE21FF31F8F5550
:105080009441E642F1499C01DC01A98FBA8F329527
:105090002295307F3227207F3227220F331F8F0146
:1050A0006F01012F1127069506950695022B132BEC
:1050B000960132952295307F3227207F3227220FAA
:1050C000331FAB2FBB27A695A695A695A22BB32B76
:1050D00095013695279536952795C401982F929579
:1050E000907F8827990F990F822B932BFC013C010D
:1050F000698A7A8AE425F5258F89988DE827F9272A
:105100009694879496948794C501982F9295907F52
:105110008827990F990F882999295C012C014F86BE
:10512000588AA224B324AE24BF248B859C85E80F23
:10513000F91F8B899C89A81EB91E0FB62D962EAD1E
:105140003FAD2D970FBE0FB66B968EAD9FAD6B9793
:105150000FBE282739278FA998AD282739270FB6E2
:1051600023968EAD9FAD23970FBE28273927C901FF
:10517000880F991F6DA97EA94D8D5E8D64277527B7
:105180000FB661964EAD5FAD61970FBE6427752770
:105190000FB625964EAD5FAD25970FBE64277527D8
:1051A000AB01452F42954F7055274695469546953C
:1051B000482B592B0FB62B964EAF5FAF2B970FBED8
:1051C000660F771FC901892F82958F709927869561
:1051D00086958695862B972B0FB62D968EAF9FAF13
:1051E0002D970FBEE40FF51F9501281F391FE00F03
:1051F000F11F2A1F3B1FEF55F44126423149AF01F1
:10520000EB8BFC8B52954295507F5427407F54275F
:10521000440F551FC9015901892F992786958695F5
:105220008695842B952BA50152954295507F542746
:10523000407F5427440F551FEF2FFF27E695E69533
:10524000E695E42BF52B6F89788DAB015695479544
:10525000569547959701322F3295307F2227330F8D
:10526000330F242B352BD90119012B863C86A6251B
:10527000B725898C9A8CA825B925F694E794F694DD
:10528000E7948B01102F1295107F0027110F110F3B
:105290000E291F290F8B188F042515250C251D2578
:1052A0004FA558A92FA138A5422753270FB66596B9
:1052B0002EAD3FAD65970FBE422753270FB62796F9
:1052C0002EAD3FAD27970FBE422753277A01440FDB
:1052D000551F0FB667962EAD3FAD67970FBE6BA9F2
:1052E0007CA9262737270FB62F966EAD7FAD2F9757
:1052F0000FBE2627372769A97AA926273727B9019C
:10530000672F62956F707727669566956695642B13
:10531000752B6DAB7EAB220F331FA701452F429536
:105320004F705527469546954695422B532B4FA7D0
:1053300058AB2D853E85260F371F69857A85641FFA
:10534000751F2A0F3B1F601F711F280F391F6E1F0B
:105350007F1F2F55344166427149C9013901929529
:105360008295907F9827807F9827880F991FFB014F
:10537000EF2FFF27E695E695E695E82BF92BCB0175
:1053800092958295907F9827807F9827880F991F04
:10539000D301AB2FBB27A695A695A695A82BB92B15
:1053A000A4015695479556954795C601982F929515
:1053B000907F8827990F990F842B952B8C012C01B6
:1053C000022513252B883C8802251325D694C794E3
:1053D000D694C794C401982F9295907F8827990FEF
:1053E000990F8C299D29898F9A8F7C01CF88D88C21
:1053F000EC24FD24EA24FB240FB66B964EAD5FAD82
:105400006B970FBE8DA59EA54827592789AD9AADEC
:10541000482759270FB629968EAD9FAD29970FBE05
:10542000482759274A01440F551F2D8D3E8D0FB631
:1054300063968EAD9FAD63970FBE282739278BAD3E
:105440009CAD282739278DA19EA128273927C9017E
:10545000892F82958F709927869586958695842BBE
:10546000952B0FB667968EAF9FAF67970FBE220F33
:10547000331FA401452F42954F70552746954695F9
:105480004695422B532B0FB66B964EAF5FAF6B9783
:105490000FBE29893A89280F391F8F859889841F63
:1054A000951F200F311F8E1D9F1D2E0F3F1F8A1F1E
:1054B0009B1F2F55344186429149A9018901098BCF
:1054C0001A8B52954295507F5427407F5427440FA2
:1054D000551FDC014C01AB2FBB27A695A695A695C1
:1054E000A42BB52BA40152954295507F5427407FA1
:1054F0005427440F551F012F112706950695069531
:10550000042B152B9101A901569547955695479562
:10551000C501982F9295907F8827990F990F842B1A
:10552000952BAC0149865A8644255525462157219D
:10553000FC017C01E421F521E427F527B694A7942A
:10554000B694A794322F3295307F2227330F330F32
:105550002A293B292B8B3C8BA901A98CBA8C4A2583
:105560005B25462357232A213B2124273527EA0F91
:10557000FB1F201F311F8FA198A50FB66D964EAD52
:105580005FAD6D970FBE842795274F8D58A1842757
:1055900095270FB62B964EAD5FAD2B970FBE842788
:1055A0009527AC01440F551F0BA91CA9AB8DBC8DD1
:1055B0000A271B27ADADBEAD0A271B270FB62D96B8
:1055C000AEADBFAD2D970FBE0A271B27D801AB2F5D
:1055D000A295AF70BB27A695A695A695A42BB52B33
:1055E000AD8FBE8F000F111FAC01452F42954F703C
:1055F0005527469546954695402B512B4FA358A7C6
:105600008B859C858A0F9B1FD601A41FB51F8E0F0B
:105610009F1FA21FB31F84529344A44EB047AC01F6
:105620001C0152954295507F5427407F5427440FC8
:10563000551F9D016D01232F33272695269526950D
:10564000242B352BA60152954295507F5427407F3D
:105650005427440F551F8101012F112706950695E8
:105660000695042B152BA3015695479556954795FE
:10567000CB01982F9295907F8827990F990F842BB3
:10568000952BAC01F701ED8BFE8B4E275F27A98888
:10569000BA884A215B217C012C01EE22FF22E426FC
:1056A000F5267695679576956795F301FE2FF29529
:1056B000F07FEE27FF0FFF0FE62BF72BED87FE871E
:1056C000AF016B897C894627572748215921E6235A
:1056D000F723E427F52789859A85E80EF91E898D39
:1056E0009A8DE81FF91F4DA55EA50FB669968EAD80
:1056F0009FAD69970FBE482759270FB621968EADEB
:105700009FAD21970FBE482759278DA99EA94827ED
:105710005927CA01BA01880F991F0FB66396AEAD1B
:10572000BFAD63970FBE4BA55CA5A427B52749A1C4
:105730005AA1A427B5274FA558A9A427B527AD017D
:10574000452F42954F705527469546954695482BCF
:10575000592B0FB663964EAF5FAF63970FBEAA0F7C
:10576000BB1FCB01892F82958F70992786958695CF
:1057700086958A2B9B2B8DA79EA7B701640F751F5B
:10578000E81FF91F620F731FE01FF11F645273447B
:10579000E44EF0479B016F8B788F32952295307FD6
:1057A0003227207F3227220F331FCF01892F9927DD
:1057B000869586958695822B932BAF0152954295BF
:1057C000507F5427407F5427440F551F9B01232FA0
:1057D0003327269526952695242B352BA5015695FE
:1057E000479556954795B401762F7295707F662739
:1057F000770F770F642B752B698F7A8FAB01442558
:105800005525422153217B01E420F520E426F5268D
:105810009694879496948794A501542F5295507F1F
:105820004427550F550F482959293A016D857E8522
:10583000462757274C215D21830106231723042780
:1058400015270FB66D96AEADBFAD6D970FBE4BA1D0
:105850005CA1A427B5270FB623964EAD5FAD239765
:105860000FBEA427B5270FB667964EAD5FAD6797FD
:105870000FBEA427B527AD01440F551FAB8CBC8CC0
:1058800069A57AA5A626B7260FB625966EAD7FAD7B
:1058900025970FBEA626B7260FB66B966EAD7FADC9
:1058A0006B970FBEA626B726B501672F62956F705E
:1058B0007727669566956695642B752B6BAB7CABED
:1058C000AA0CBB1CAB2FA295AF70BB27A695A695C3
:1058D000A695AA29BB290FB66D96AEAFBFAF6D973F
:1058E0000FBE4D895E89460F571F6B897C896A1FE1
:1058F0007B1F4E0D5F1D601F711F480F591F621FD8
:10590000731F44525344644E7047CA014D8B5E8BE3
:1059100092958295907F9827807F9827880F991F6E
:105920009B014B01232F3327269526952695282B5F
:10593000392BC40192958295907F9827807F982774
:10594000880F991F452F5527469546954695482B14
:10595000592BC1019695879596958795D601BA2FB3
:10596000B295B07FAA27BB0FBB0FA82BB92BCD01D7
:10597000E98CFA8C8E259F250F89188D8023912321
:105980008D010E211F2108271927D694C794D6947C
:10599000C794C101982F9295907F8827990F990FEE
:1059A0008C299D297C01EB86FC86698A7A8A86256A
:1059B00097258E239F23E620F720E826F9260FB6A9
:1059C0006996AEACBFAC69970FBE8FA998ADA826FB
:1059D000B9260FB627968EAD9FAD27970FBEA82686
:1059E000B9268D8D9E8DA826B926C501880F991FD1
:1059F0002BA43CA40FB661966EAD7FAD61970FBE30
:105A00002626372669A97AA9262637266FA178A5E2
:105A100026263726B101672F62956F707727669526
:105A200066956695682B792B6BA77CA7220C331C97
:105A3000C501892F82958F709927869586958695C1
:105A4000822993290FB669968EAF9FAF69970FBED3
:105A5000460E571E6D857E85681F791FC201800F17
:105A6000911F6E1D7F1D820F931F641F751F84522F
:105A700093449C01644E704789010D871E8792955F
:105A80008295907F9827807F9827880F991FAB0178
:105A90002B01452F5527469546954695482B592B62
:105AA000C20192958295907F9827807F9827880FD2
:105AB000991F012F1127069506950695082B192B7E
:105AC000CF88D88CC6019695879596958795BF0106
:105AD000762F7295707F6627770F770F682B792B5B
:105AE000CB018A279B27ED88FE888E219F219B0171
:105AF0005B012A233B2328273927F695E795F6955E
:105B0000E795B601762F7295707F6627770F770F2E
:105B10006E2B7F2BCB016B847C8486259725882177
:105B20009921FB011B01E621F721E827F927240F22
:105B3000351FE01FF11F4BA15CA10FB665968EAD1E
:105B40009FAD65970FBE482759270FB629968EAD92
:105B50009FAD29970FBE482759270FB663968EAD84
:105B60009FAD63970FBE48275927CA01BA01880F16
:105B7000991F09A51AA50FB62F964EAD5FAD2F97A9
:105B80000FBE042715274DA15EA1042715274DA59B
:105B90005EA504271527A801452F42954F7055276C
:105BA000469546954695482B592B49A75AA7000F6D
:105BB000111FCB01892F82958F7099278695869525
:105BC0008695802B912B8BA39CA3698D7A8D640F76
:105BD000751F49895A89481F591F620F731F4E1F2D
:105BE0005F1F64527344444E5047CB01698F7A8FD4
:105BF00092958295907F9827807F9827880F991F8C
:105C00008A016A01012F1127069506950695082B32
:105C1000192BC60192958295907F9827807F9827AF
:105C2000880F991FAB01452F5527469546954695F8
:105C3000482B592BB701CB0196958795969587955B
:105C4000F401FE2FF295F07FEE27FF0FFF0FE82BF8
:105C5000F92BE98BFA8BCF01AB8EBC8E8A259B2565
:105C6000ED84FE848E219F21EA21FB21E827F9277C
:105C700096948794969487949B01322F3295307F27
:105C80002227330F330F28293929C90159018225C9
:105C90009325842195212221332128273927EA0FB2
:105CA000FB1F261D371D6FA978AD89AD9AAD6827FA
:105CB00079270FB62B968EAD9FAD2B970FBE682719
:105CC00079278BA99CA968277927CB014B01880FDD
:105CD000991F0FB66196AEADBFAD61970FBE6BADAC
:105CE0007CADA627B7270FB62D966EAD7FAD2D974D
:105CF0000FBEA627B7270FB66D966EAD7FAD6D9719
:105D00000FBEA627B727BD01672F62956F70772753
:105D1000669566956695682B792B0FB661966EAF82
:105D20007FAF61970FBEAA0FBB1FC401892F829559
:105D30008F7099278695869586958A2B9B2B8FAB9E
:105D400098AFE60FF71F281F391FE00FF11F241F20
:105D5000351FE452F344244E3047AF01EF87F88BF0
:105D600052954295507F5427407F5427440F551F2A
:105D7000C901892F9927869586958695842B952B21
:105D8000B90172956295707F7627607F7627660FDE
:105D9000771FAF01452F5527469546954695462BCB
:105DA000572BB7017695679576956795F201FE2F8B
:105DB000F295F07FEE27FF0FFF0FE62BF72BEB8B13
:105DC000FC8BDF0109891A89A027B127698C7A8C9D
:105DD000A621B721BF01602371236A277B27569430
:105DE000479456944794F701FE2FF295F07FEE27E3
:105DF000FF0FFF0FE429F5298F010D871E87D801BA
:105E0000AD8ABE8AAA25BB25AC21BD210A211B2152
:105E10000A271B270FB66596AEADBFAD65970FBEBF
:105E2000EF8DF8A1AE27BF27EDA9FEA9AE27BF27AA
:105E3000EBA5FCA5AE27BF277D01AA0FBB1F0FB6A0
:105E40002F96AEACBFAC2F970FBEEDADFEADAE261C
:105E5000BF26EFA5F8A9AE26BF260FB66996EEAD10
:105E6000FFAD69970FBEAE26BF26F501EF2FE29575
:105E7000EF70FF27E695E695E695EA2BFB2B0FB62C
:105E80002F96EEAFFFAF2F970FBEAA0CBB1CD7010A
:105E9000AB2FA295AF70BB27A695A695A695AA296C
:105EA000BB290FB66596AEAFBFAF65970FBEEB8C43
:105EB000FC8CEE0EFF1E2A1E3B1EF701E60FF71F9D
:105EC000D101A01FB11FE80FF91FA41FB51FE45295
:105ED000F344A44EB047CF01AF014B8F5C8F929536
:105EE0008295907F9827807F9827880F991FBD0102
:105EF0004D01672F7727669566956695682B792BF8
:105F0000C40192958295907F9827807F9827880F6B
:105F1000991F452F5527469546954695482B592B51
:105F20007301D701B695A795B695A795C601982F89
:105F30009295907F8827990F990F8A2B9B2BDC01D4
:105F4000EB89FC89AE27BF276F847888A621B7210B
:105F50008C010E231F230A271B27D694C794D6949F
:105F6000C794F701FE2FF295F07FEE27FF0FFF0F8A
:105F7000EC29FD292F01D201CD84DE84AC25BD257D
:105F8000A223B3237201EC20FD20EA26FB26A9AD53
:105F9000BAAD0FB62196EEADFFAD21970FBEAE277D
:105FA000BF270FB66796EEADFFAD67970FBEAE2762
:105FB000BF27E9A5FAA5AE27BF275D01AA0FBB1F22
:105FC0002BAC3CACE9A1FAA12E263F260FB66B966E
:105FD000EEADFFAD6B970FBE2E263F26EBA1FCA1C9
:105FE0002E263F26F101EF2FE295EF70FF27E69571
:105FF000E695E695EA2BFB2BEBAFFCAF220C331CAE
:10600000D501AB2FA295AF70BB27A695A695A695F7
:10601000A229B329A9AFBAAFA988BA88AE0EBF1E0C
:106020002D883E882A1E3B1EF501E00FF11FD1018D
:10603000AE1DBF1DE60FF71FA41FB51FE452F344AA
:10604000A44EB047AF0152954295507F5427407FF0
:106050005427440F551FBD015D01672F77276695B3
:1060600066956695642B752BA50152954295507FD8
:106070005427407F5427440F551F8F011F01012FC4
:106080001127069506950695042B152BA301569509
:10609000479556954795F901FE2FF295F07FEE272B
:1060A000FF0FFF0FE42BF52BEF8BF88FDF01A827F5
:1060B000B927EB8CFC8CAE21BF21AF0148235923BB
:1060C0004A275B273695279536952795F301FE2FAE
:1060D000F295F07FEE27FF0FFF0FE22BF32BEF87F8
:1060E000F88BDF01A425B525A821B9219F01242122
:1060F00035212A273B27460F571F201F311FAF8D01
:10610000B8A10FB623966EAD7FAD23970FBEA6271D
:10611000B7276D8D7E8DA627B7270FB661966EAD1A
:106120007FAD61970FBEA627B727BD01660F771F0A
:10613000EDADFEAD0FB625960EAD1FAD25970FBE8A
:10614000E027F1270FA118A5E027F1270FA918AD27
:10615000E027F1278F01012F02950F701127069577
:1061600006950695062B172B0DAF1EAFEE0FFF1FE2
:10617000AB2FA295AF70BB27A695A695A695AE2B83
:10618000BF2BAF8FB8A36B897C89600F711FF6019D
:10619000EA1FFB1F640F751FE21FF31F6452734455
:1061A000E44EF0479B01AB014B8B5C8B3295229503
:1061B000307F3227207F3227220F331F8F016F015C
:1061C000012F1127069506950695022B132B960194
:1061D00032952295307F3227207F3227220F331FBE
:1061E000452F5527469546954695422B532BD7016B
:1061F0009D013695279536952795B401762F729592
:10620000707F6627770F770F622B732B9B01EF89C7
:10621000F88D2E273F27222133217B013B01EE22DF
:10622000FF22E226F3269694879496948794BD01E4
:10623000762F7295707F6627770F770F68297929F7
:106240009B014B01EF85F8892E273F272A213B210F
:106250006E237F2362277327E80EF91E641D751DC8
:106260000FB621962EAD3FAD21970FBE0FB62796E4
:106270008EAD9FAD27970FBE282739270FB663969F
:106280008EAD9FAD63970FBE282739270FB62F9687
:106290008EAD9FAD2F970FBE28273927C901880FD4
:1062A000991FE9A1FAA1A9A9BAA9EA27FB27ADA5D7
:1062B000BEA5EA27FB270FB66596AEADBFAD6597C5
:1062C0000FBEEA27FB27DF01AB2FA295AF70BB27DC
:1062D000A695A695A695A82BB92BA9A3BAA3EE0FB0
:1062E000FF1F232F22952F7033272695269526955D
:1062F0002E2B3F2B0FB621962EAF3FAF21970FBE0F
:10630000C7018A0F9B1F621F731F800F911F641F9D
:10631000751F84529344644E70479C01AC014D87B5
:106320005E8732952295307F3227207F3227220FD9
:10633000331FCB01892F9927869586958695822BC9
:10634000932B9B0132952295307F3227207F322775
:10635000220F331F452F5527469546954695422BCC
:10636000532BD1019D013695279536952795F5013B
:10637000FE2FF295F07FEE27FF0FFF0FE22BF32B9E
:10638000E98FFA8F9F011301222533254B885C8802
:10639000242135217F01E220F320E226F326B69462
:1063A000A794B694A7949D01322F3295307F22276F
:1063B000330F330F2A293B29F9018B8E9C8E282518
:1063C00039252C213D218F015F0108211921022748
:1063D00013270FB623962EAD3FAD23970FBE0FB6F2
:1063E0002996EEADFFAD29970FBE2E273F27EBA9CB
:1063F000FCA92E273F27EBADFCAD2E273F27D90167
:10640000AA0FBB1F0FB625968EAC9FAC25970FBE6B
:10641000EDA1FEA18E269F260FB66D96EEADFFADC7
:106420006D970FBE8E269F26E9ADFAAD8E269F266C
:10643000F401EF2FE295EF70FF27E695E695E695DC
:10644000EA2BFB2B0FB62596EEAFFFAF25970FBEBD
:10645000880C991C232F22952F703327269526957B
:106460002695282939290FB623962EAF3FAF2397BB
:106470000FBEAF89B88DAE0FBF1FEF85F889E21F41
:10648000F31FAE0DBF1DE01FF11FA80FB91FE41FC2
:10649000F51FA452B344E44EF047CD01AD014F8B3C
:1064A000588F92958295907F9827807F9827880FA4
:1064B000991FDF014F01AB2FBB27A695A695A69587
:1064C000A82BB92B940132952295307F3227207F5B
:1064D0003227220F331FCA01892F99278695869567
:1064E0008695822B932B72019701369527953695C9
:1064F0002795A601542F5295507F4427550F550FCD
:10650000422B532B9A01E98DFA8D2E273F276D845C
:106510007E84262137218A010E231F230227132779
:10652000D694C794D694C7949701322F3295307F72
:106530002227330F330F2C293D292901A98ABA8A32
:106540002A253B25262337237201EA20FB20E22659
:10655000F3260FB627962EAD3FAD27970FBE0FB689
:106560002B96EEADFFAD2B970FBE2E273F27EBA549
:10657000FCA52E273F27EDADFEAD2E273F27690155
:10658000220F331FA9A8BAA80FB62D96EEADFFAD06
:106590002D970FBEAE26BF260FB66996EEADFFADA6
:1065A00069970FBEAE26BF26EF8DF8A1AE26BF2697
:1065B000F501EF2FE295EF70FF27E695E695E6955A
:1065C000E22BF32BE9ABFAABAA0CBB1C9601232FF1
:1065D00022952F7033272695269526952A293B2923
:1065E0000FB627962EAF3FAF27970FBE2E0E3F1E3A
:1065F000EB8DFC8DE21FF31F9101200F311FEE1D6B
:10660000FF1D2A0F3B1FE81FF91F24523344E44E9D
:10661000F047C90192958295907F9827807F9827AF
:10662000880F991FDF015F01AB2FBB27A695A695A9
:10663000A695A82BB92BC50192958295907F982796
:10664000807F9827880F991F89011901012F112731
:10665000069506950695082B192B7301C70196958B
:10666000879596958795FB01FE2FF295F07FEE2793
:10667000FF0FFF0FE82BF92BEF87F88B9F012427E3
:1066800035276F88788C26213721CF0184239523E5
:106690008227932776956795769567959701322F90
:1066A0003295307F2227330F330F262B372B2D8740
:1066B0003E87B9016425752568217921242135217A
:1066C000262737278A0F9B1F201F311F0FB62996B9
:1066D000AEADBFAD29970FBE6DA97EA9A627B7277E
:1066E00069A57AA5A627B72769A17AA1A627B72702
:1066F000BD01660F771FEDA0FEA0EFA5F8A9EE265D
:10670000FF26EBA1FCA1EE26FF260FB62196EEADEB
:10671000FFAD21970FBEEE26FF268701012F0295C0
:106720000F701127069506950695062B172B0DA3BE
:106730001EA3EE0CFF1CAB2FA295AF70BB27A69536
:10674000A695A695AE29BF290FB62996AEAFBFAFC5
:1067500029970FBE698D7A8D600F711FE989FA89BB
:10676000EA1FFB1F680F791FE21FF31F6452734477
:10677000E44EF0479B01DB01A98FBA8F3295229539
:10678000307F3227207F3227220F331FCF016F0146
:10679000892F9927869586958695822B932BB6010E
:1067A00072956295707F7627607F7627660F771FD8
:1067B0009D01232F3327269526952695262B372BAB
:1067C0008301B8017695679576956795F401FE2F5C
:1067D000F295F07FEE27FF0FFF0FE62BF72BBF019F
:1067E000EF84F8886E257F25310166217721DF014E
:1067F0001F01AE21BF21A627B727969487949694B0
:106800008794B801762F7295707F6627770F770F80
:10681000682979298B01ED84FE846E257F256A2104
:106820007B21F8014801EE21FF21E627F727A40F7D
:10683000B51FE41DF51D0FB62B966EAD7FAD2B97E2
:106840000FBE0FB667964EAD5FAD67970FBE64275C
:1068500075270FB661964EAD5FAD61970FBE642789
:1068600075270FB625964EAD5FAD25970FBE6427F1
:106870007527AB01440F551F0FB62D96EEACFFAC3C
:106880002D970FBE0FB66B960EAD1FAD6B970FBE5B
:10689000E026F1260FA918ADE026F1260FB62396C3
:1068A0000EAD1FAD23970FBEE026F1268701012F05
:1068B00002950F701127069506950695042B152B4A
:1068C0000FB62D960EAF1FAF2D970FBEEE0CFF1C0F
:1068D000672F62956F7077276695669566956E2926
:1068E0007F290FB62B966EAF7FAF2B970FBEA00FF1
:1068F000B11FE61FF71FA80FB91FE21FF31FA45215
:10690000B344E44EF0479D0132952295307F322703
:10691000207F3227220F331FCF01892F9927869599
:1069200086958695822B932BAF0152954295507F89
:106930005427407F5427440F551F9D01232F332791
:10694000269526952695242B352B7301A701569560
:106950004795569547958501102F1295107F002772
:10696000110F110F042B152B0B8F1C8FB801A101D8
:106970004D8B5E8B64277527298C3A8C622173219D
:1069800038016422752266267726B694A794B694B9
:10699000A7948701102F1295107F0027110F110F58
:1069A0000A291B290B8B1C8BB8018F8A988E6825AE
:1069B00079256C217D2108211921062717276DA92A
:1069C0007EA94D8D5E8D642775270FB62F964EAD2F
:1069D0005FAD2F970FBE6427752749A95AA9642771
:1069E00075274B01660F771FEFA4F8A84FA158A594
:1069F000E426F5260FB665964EAD5FAD65970FBEE2
:106A0000E426F5260FB627964EAD5FAD27970FBE4D
:106A1000E426F526A701452F42954F705527469548
:106A200046954695462B572B4FA758ABEE0CFF1CAF
:106A3000B401672F62956F707727669566956695A6
:106A40006E297F296DAB7EABEF84F888E40EF51ECE
:106A5000AD84BE84A61EB71EA701460D571DB50105
:106A6000601F711F480F591F621F731F4452534408
:106A7000644E70479A015A0132952295307F322731
:106A8000207F3227220F331FCB012B01892F99271B
:106A9000869586958695822B932BA20152954295D9
:106AA000507F5427407F5427440F551F9501AF86D0
:106AB000B88A232F3327269526952695242B352B08
:106AC000B1017695679576956795A601542F5295F5
:106AD000507F4427550F550F462B572BBA010B8D6E
:106AE0001C8D602771276A237B233A016022712263
:106AF00066267726D694C794D694C794B101762F8C
:106B00007295707F6627770F770F6C297D297B013F
:106B1000E98EFA8E0B891C89602771276E237F23EB
:106B2000E022F122E626F7260FB667966EAD7FAD1E
:106B300067970FBE0FB663960EAD1FAD63970FBE7E
:106B4000602771270BAD1CAD602771270DA11EA119
:106B5000602771274B01660F771F0FB66B96CEAC7F
:106B6000DFAC6B970FBE0DA51EA5C026D12609ADC3
:106B70001AADC026D1260FB629960EAD1FAD2997A6
:106B80000FBEC026D1268601012F02950F70112756
:106B9000069506950695062B172B0FB66B960EAF2E
:106BA0001FAF6B970FBECC0CDD1CB401672F629535
:106BB0006F7077276695669566956C297D290FB667
:106BC00067966EAF7FAF67970FBECD88DE88C00E29
:106BD000D11E0F89188D061F171FB601660D771D70
:106BE0000E1D1F1D680F791F021F131F645273446F
:106BF000044E1047CB0192958295907F9827807F15
:106C00009827880F991F98016801232F332726950D
:106C100026952695282B392BC60192958295907F33
:106C20009827807F9827880F991F8B011B012D8A39
:106C30003E8A012F1127069506950695082B192BDC
:106C4000CD019695879596958795BF01762F72957C
:106C5000707F6627770F770F682B792B3B016427AE
:106C600075276A217B21C3018423952386279727D3
:106C7000F695E795F695E795BA2FB295B07FAA27D6
:106C8000BB0FBB0FAE2BBF2B4D01B401A98DBA8D2D
:106C90006A277B2764217521F401EA23FB23E62779
:106CA000F727820F931FE01FF11F6D8D7E8D2BA99B
:106CB0003CA9622773272DAD3EAD622773270FB61F
:106CC0002D962EAD3FAD2D970FBE622773279B01EA
:106CD000220F331FEFA0F8A40FB66D96AEADBFAD77
:106CE0006D970FBEEA26FB260F8D18A1E026F12630
:106CF0000FB62B96AEADBFAD2B970FBEEA26FB2687
:106D00008701012F02950F701127069506950695AC
:106D1000022B132B0FA318A7EE0CFF1C672F6295F5
:106D20006F7077276695669566956E297F296D8FBA
:106D30007E8F2B8D3C8D200F311F0B891C89061FE8
:106D4000171F280F391F0E1F1F1F24523344044ED4
:106D50001047C901F901EB8FFC8F92958295907FC6
:106D60009827807F9827880F991F98015801232F13
:106D70003327269526952695282B392BB501729514
:106D80006295707F7627607F7627660F771FCF0129
:106D9000892F9927869586958695862B972B0F8523
:106DA0001889B8017695679576956795D201BA2FBF
:106DB000B295B07FAA27BB0FBB0FA62BB72BAB8B0F
:106DC000BC8BBD016625772562217321A621B721E1
:106DD000A627B7275694479456944794B801762F20
:106DE0007295707F6627770F770F64297529FB01ED
:106DF0001B018F8A988EE825F925EC21FD21682159
:106E000079216E277F27A40FB51F498D5A8D641FE6
:106E1000751F0FB66396EEADFFAD63970FBE4BA522
:106E20005CA5E427F52749A15AA1E427F5274FA53A
:106E300058A9E427F527AF01440F551FEDA4FEA480
:106E40000FB669960EAD1FAD69970FBEE026F1260D
:106E50000FB621960EAD1FAD21970FBEE026F1268D
:106E60000DA91EA9E026F1268701012F02950F70BA
:106E70001127069506950695042B152B0DA71EA721
:106E8000EE0CFF1CEF2FE295EF70FF27E695E695DD
:106E9000E695EE29FF290FB66396EEAFFFAF639735
:106EA0000FBEA00FB11F6E1F7F1FA20FB31F681F61
:106EB000791FA452B344644E7047CD01AF83B887A5
:106EC00092958295907F9827807F9827880F991FA9
:106ED0009B01232F3327269526952695282B392B82
:106EE000AB0152954295507F5427407F5427440F61
:106EF000551FCD01892F9927869586958695842BD8
:106F0000952B0D891E89A80156954795569547954D
:106F1000F601FE2FF295F07FEE27FF0FFF0FE42B17
:106F2000F52BE98BFA8BAF01AB89BC894A275B272C
:106F30004B8C5C8C442155217F01EA22FB22E42604
:106F4000F526D694C794D694C794A801542F529589
:106F5000507F4427550F550F4C295D29FA01ED8BC1
:106F6000FE8B422553254A215B21E221F321E427B0
:106F7000F5274BA95CA9A9A5BAA54A275B270FB697
:106F800025960EAD1FAD25970FBE402751270FB692
:106F90006B96AEADBFAD6B970FBE4A275B274A011C
:106FA000440F551F0FB66D96CEACDFAC6D970FBE7C
:106FB000ABA1BCA1CA26DB260FB623960EAD1FAD32
:106FC00023970FBEC026D1260FB66796AEADBFADD4
:106FD00067970FBECA26DB268601012F02950F7028
:106FE0001127069506950695042B152BA801498FA8
:106FF0005A8FCC0CDD1C8401012F02950F701127D4
:107000000695069506950C291D290BAB1CAB640E45
:10701000751EAF89B88DA01FB11FA3014E0D5F1D56
:10702000AE1FBF1F420F531FA81FB91F4452534426
:10703000A44EB047CA01FA01E987FA879295829572
:10704000907F9827807F9827880F991F9D01232F75
:107050003327269526952695282B392BAD01529559
:107060004295507F5427407F5427440F551FCF012E
:10707000892F9927869586958695842B952B820155
:10708000F801F695E795F695E795A501542F5295E9
:10709000507F4427550F550F4E2B5F2BFA018988DF
:1070A0009A88E825F9254F805884E421F5216A0162
:1070B000C820D920CE26DF26B694A794B694A794EC
:1070C000F801FE2FF295F07FEE27FF0FFF0FEA2960
:1070D000FB297F01EB8EFC8E0D891E89E027F127AD
:1070E000E623F723E022F122EE26FF26EBA5FCA5FE
:1070F0000FB661960EAD1FAD61970FBEE027F12769
:1071000009A91AA9E027F1270FA118A5E027F1275F
:107110003F01EE0FFF1F0FB66996AEACBFAC69978B
:107120000FBE0FA918ADA026B1260FB627960EAD3B
:107130001FAD27970FBEA026B1260D8D1E8DA02650
:10714000B1268501012F02950F701127069506952E
:1071500006950E2B1F2BF801EF8BF88FAA0CBB1C8A
:107160008301012F02950F7011270695069506954C
:107170000A291B290BA71CA7AB88BC88AE0EBF1E13
:10718000201E311EF501EC0DFD1D81010E1D1F1D80
:10719000E20FF31F081F191FE452F344044E104777
:1071A000CF017F0192958295907F9827807F9827C5
:1071B000880F991F98016801232F3327269526955C
:1071C0002695282B392BC60192958295907F98277A
:1071D000807F9827880F991F3701EF2FFF27E695AB
:1071E000E695E695E82BF92B7201C70196958795F0
:1071F000969587958B01102F1295107F0027110F00
:10720000110F082B192BC8015801AB86BC868427A7
:10721000952729843A8482259325769567957695D6
:1072200067958701102F1295107F0027110F110FFE
:10723000062B172BB80128014F8258860B8D1C8D09
:10724000602771276A277B27820F931F6E1F7F1F7E
:10725000E9A5FAA50FB62F962EAD3FAD2F970FBE1D
:10726000E227F3272DA13EA1E227F3272DA53EA576
:10727000E227F3279F01220F331FEBA0FCA00FB6DC
:1072800065960EAD1FAD65970FBEE026F1260FB6D1
:1072900029960EAD1FAD29970FBEE026F1260FB639
:1072A00063960EAD1FAD63970FBEE026F1268701F2
:1072B000012F02950F701127069506950695022B52
:1072C000132B0BA31CA3EE0CFF1CEF2FE295EF700A
:1072D000FF27E695E695E695EE29FF29E9A7FAA7A7
:1072E000800E911E0D891E890E1F1F1FF401E80FCD
:1072F000F91F061F171FEA52FE430D4915439F0150
:10730000BF01698B7A8B32952295307F3227207F9F
:107310003227220F331FC8014801892F99278695EC
:1073200086958695822B932B940132952295307FFA
:107330003227207F3227220F331F672F772766954A
:1073400066956695622B732B71019701369527958B
:1073500036952795FD01FE2FF295F07FEE27FF0F62
:10736000FF0FE22BF32B8F011F012D8A3E8A0A2586
:107370001B2553010A251B25B695A795B695A795FC
:107380009701322F3295307F2227330F330F2A2B6C
:107390003B2BD901390169867A86A425B525AC2510
:1073A000BD25040F151F2B8D3C8DA21FB31F0FB6DB
:1073B00061964EAD5FAD61970FBE2BAD3CAD4227E0
:1073C00053270FB62D962EAD3FAD2D970FBE4227FA
:1073D0005327298D3A8D422753279A01220F331FB5
:1073E000EFA8F8ACE9ADFAADEE26FF260FB62B9666
:1073F000EEADFFAD2B970FBEEE26FF26EBA9FCA945
:10740000EE26FF26F701EF2FE295EF70FF27E695B6
:10741000E695E695E22BF32BED87FE87EE0CFF1C3D
:10742000452F42954F7055274695469546954E29CE
:107430005F290FB661964EAF5FAF61970FBE0E0F1B
:107440001F1FA41FB51F080F191FA61FB71F0A5221
:107450001E43AD49B5439801A8010FB669964EAFDA
:107460005FAF69970FBE32952295307F3227207F1C
:107470003227220F331FCD01892F992786958695B4
:107480008695822B932B9D0132952295307F322752
:10749000207F3227220F331F452F552746954695CB
:1074A0004695422B532B9501369527953695279572
:1074B000B601762F7295707F6627770F770F622B54
:1074C000732B0FB66D966EAF7FAF6D970FBE7B01BE
:1074D000E224F32449885A88E424F524D694C794F6
:1074E000D694C794B501762F7295707F6627770F73
:1074F000770F6C297D296B8B7C8B6625772568251A
:1075000079250FB62F962EAD3FAD2F970FBEEDAD5F
:10751000FEAD2E273F27EFA5F8A92E273F27EF899D
:10752000F88D2E273F276901220F331F0FB665966E
:10753000AEACBFAC65970FBEEF8DF8A1AE26BF26EF
:10754000EDA9FEA9AE26BF26EBA5FCA5AE26BF265B
:10755000F501EF2FE295EF70FF27E695E695E695AA
:10756000E22BF32BEF87F88BAA0CBB1C9601232F81
:1075700022952F7033272695269526952A293B2973
:107580000FB62F962EAF3FAF2F970FBE0B851C85E2
:107590000E0F1F1FEF81F885E21FF31F98012E0DBC
:1075A0003F1DE61FF71F280F391FE41FF51F2A5242
:1075B0003E431901ED49F54332952295307F32273C
:1075C000207F3227220F331F8F013F01012F112708
:1075D000069506950695022B132B9301329522955D
:1075E000307F3227207F3227220F331FA101452F02
:1075F0005527469546954695422B532BC2019C0133
:107600003695279536952795B401762F7295707F1C
:107610006627770F770F622B732B6B010FB66D9672
:107620002EAD3FAD6D970FBEC226D3260FB669961D
:107630004EAC5FAC69970FBEC424D5249694879452
:1076400096948794982F9295907F8827990F990FF9
:10765000882999297C014C01898A9A8A8B899C897D
:10766000E826F926EA26FB262BAD3CAD89A19AA196
:10767000282739270FB66B968EAD9FAD6B970FBE3F
:10768000282739278BA19CA1282739275901220FA8
:10769000331F89AD9AAD0FB62196EEADFFAD2197A0
:1076A0000FBE8E279F270FB66796EEADFFAD67978B
:1076B0000FBE8E279F27E9A5FAA58E279F27FC01DD
:1076C000EF2FE295EF70FF27E695E695E695E22B22
:1076D000F32BEB8FFC8F880F991F9501232F229599
:1076E0002F703327269526952695282B392B2BAFDF
:1076F0003CAF8D899E898E0F9F1FE985FA85E21F19
:10770000F31F9C012C0D3D1DEE1DFF1D200F311F91
:10771000E41FF51F2A523E43ED49F543C901890193
:107720000D8B1E8B92958295907F9827807F98274E
:10773000880F991F9F016F01232F332726952695C8
:107740002695282B392BA60152954295507F542718
:10775000407F5427440F551FC801892F99278695CC
:1077600086958695842B952B5201A50156954795B4
:1077700056954795FD01FE2FF295F07FEE27FF0FFE
:10778000FF0FE42BF52B7F018F010FAB18AFE6261F
:10779000F726E224F324B695A795B695A795A501FB
:1077A000542F5295507F4427550F550F4A2B5B2B72
:1077B0000FB669964EAF5FAF69970FBE4825592542
:1077C00046255725E20EF31E481F591F2DAD3EAD2D
:1077D0000FB625968EAD9FAD25970FBE282739276A
:1077E0008FA198A5282739278D859E852827392799
:1077F000C901880F991FEF8DF8A10FB62396AEAD82
:10780000BFAD23970FBEEA27FB27AD8DBE8DEA27BC
:10781000FB270FB66196AEADBFAD61970FBEEA27ED
:10782000FB27DF01AB2FA295AF70BB27A695A695CE
:10783000A695A82BB92BAF8FB8A3EE0FFF1F232F50
:1078400022952F7033272695269526952E2B3F2B94
:107850002DAF3EAF0FB66D96EEADFFAD6D970FBE7F
:10786000EA0FFB1FAB89BC89A21FB31FEE0DFF1DE2
:10787000A41FB51FEA52FE43AD49B543CF010FB671
:107880006D96EEAFFFAF6D970FBE92958295907F8C
:107890009827807F9827880F991F9D015D01232FCE
:1078A0003327269526952695282B392BA501529509
:1078B0004295507F5427407F5427440F551FCF01D6
:1078C000892F9927869586958695842B952BA101DE
:1078D0005695479556954795F301FE2FF295F07F03
:1078E000EE27FF0FFF0FE42BF52BDF012F0149AE31
:1078F0005AAEA027B1278D889E88A825B9257694F1
:10790000679476946794A101542F5295507F442731
:10791000550F550F46295729FA011A012B863C8627
:107920000FB669964EAD5FAD69970FBEE427F52798
:10793000EC25FD25A60FB71F49895A89E41FF51FBD
:1079400009A11AA149A95AA9042715274DA55EA581
:10795000042715274F85588904271527B801660F76
:10796000771F0FB62196EEACFFAC21970FBE0FB676
:1079700027964EAD5FAD27970FBEE426F5260FB6CE
:1079800063964EAD5FAD63970FBEE426F5260FB646
:107990002F964EAD5FAD2F970FBEE426F526A701BB
:1079A000452F42954F705527469546954695462B4F
:1079B000572B0FB621964EAF5FAF21970FBEEE0C3F
:1079C000FF1C012F02950F7011270695069506954D
:1079D0000E291F2909A31AA3A40FB51FE01FF11F29
:1079E000A20FB31FE81FF91FAA52BE43ED49F5438A
:1079F0009D01AB8BBC8B32952295307F3227207F47
:107A00003227220F331FCF01892F9927869586951C
:107A10008695822B932BAF0152954295507F542728
:107A2000407F5427440F551F9D01232F3327269550
:107A300026952695242B352BA401569547955695CA
:107A40004795D601BA2FB295B07FAA27BB0FBB0FBF
:107A5000A42BB52BBD013D010FB665966EAE7FAE72
:107A600065970FBE642575250FB66D964EAC5FAC5D
:107A70006D970FBE64257525D694C794D694C79488
:107A80008401102F1295107F0027110F110F0C2960
:107A90001D290D8B1E8B022513250A251B250FB6CC
:107AA00025964EAD5FAD25970FBEADA1BEA14A276D
:107AB0005B27E98CFA8C4E255F25EB8CFC8C4E25E0
:107AC0005F251A01440F551F0FB62396EEACFFAC8D
:107AD00023970FBE0FB62996AEADBFAD29970FBE47
:107AE000EA26FB26CBA8DCA8EC24FD24ABADBCAD7C
:107AF000EA26FB26D701AB2FA295AF70BB27A69530
:107B0000A695A695A42BB52BAD01498B5A8BEE0CEF
:107B1000FF1CD101AB2FA295AF70BB27A695A695F0
:107B2000A695AE29BF290FB62596AEAFBFAF259754
:107B30000FBEEFA8F8ACE40EF51E0FB66996CEACFA
:107B4000DFAC69970FBECA1EDB1EA701460F571F89
:107B5000D601A01FB11F480F591FA21FB31F4A52C1
:107B60005E43AD49B5439A01CA018FAB98AF3295D8
:107B70002295307F3227207F3227220F331FBD010D
:107B80004D01672F7727669566956695622B732B57
:107B9000A40152954295507F5427407F5427440FAB
:107BA000551F9C01232F3327269526952695242B98
:107BB000352BC201AC015695479556954795D50191
:107BC000BA2FB295B07FAA27BB0FBB0FA42BB52B42
:107BD0008D012D010FB623964EAE5FAE23970FBEDB
:107BE000062517256B887C8806251725B694A7944B
:107BF000B694A794982F9295907F8827990F990F04
:107C00008A299B297C015C010FB66D96AEAEBFAE92
:107C10006D970FBE8D899E89E826F926EE26FF26F0
:107C200049A95AA90FB62D968EAD9FAD2D970FBEBF
:107C300048275927CF88D88C4C255D25CF8CD8A0D4
:107C40004C255D25DA01440F551F0FB62796CEACA3
:107C5000DFAC27970FBE0FB62B968EAD9FAD2B973F
:107C60000FBEC826D9262BA43CA4C224D3248DAD94
:107C70009EADC826D926C601892F82958F70992777
:107C8000869586958695842B952B89879A87CC0C2B
:107C9000DD1CAB2FA295AF70BB27A695A695A69528
:107CA000AC29BD29A9ABBAAB49AD5AAD480F591F94
:107CB0008B859C858A1F9B1F400F511F8E1D9F1D0A
:107CC000460F571F821F931F4A525E438D499543AB
:107CD0007C01CA018A0109AF1AAF92958295907F03
:107CE0009827807F9827880F991F9701232F332784
:107CF000269526952695282B392BC7019295829596
:107D0000907F9827807F9827880F991F012F112730
:107D1000069506950695082B192BB301CB01969570
:107D2000879596958795AF01542F5295507F44279C
:107D3000550F550F482B592BCA013A010FB66996BA
:107D40006EAE7FAE69970FBE84259525CFA8D8ACBF
:107D50008C259D25F695E795F695E795AB01542F73
:107D60005295507F4427550F550F4E2B5F2B1A010C
:107D70002B8A3C8A4A255B2548255925820F931F6B
:107D8000401F511FEDA1FEA12FA538A9E227F3271F
:107D90002BA13CA1E227F3270FB621962EAD3FADD4
:107DA00021970FBEE227F3279F01DF01220F331F28
:107DB0000FB62996EEADFFAD29970FBE6DA97EA92E
:107DC000E627F72709A51AA5E027F12769A17AA1D7
:107DD000E627F7278F01012F02950F7011270695CF
:107DE00006950695022B132B0B871C87EE0FFF1FA2
:107DF000AB2FA295AF70BB27A695A695A695AE2BE7
:107E0000BF2BADA3BEA30FB665966EAD7FAD6597D4
:107E10000FBE600F711FED89FE89EA1FFB1F680FFF
:107E2000791FE41FF51F6A527E43ED49F5439B011C
:107E30008B010FB665960EAF1FAF65970FBE3295DB
:107E40002295307F3227207F3227220F331FCF0128
:107E50005F01892F9927869586958695822B932B8E
:107E6000950132952295307F3227207F3227220FCD
:107E7000331F012F1127069506950695022B132B0C
:107E8000B6019B013695279536952795D401BA2FD3
:107E9000B295B07FAA27BB0FBB0FA22BB32BAD8B24
:107EA000BE8BA625B725C9ACDAACAC25BD2596940A
:107EB0008794969487949B01322F3295307F2227A6
:107EC000330F330F28293929390129014FAA58AE18
:107ED000622473246E247F240FB623962EAD3FAD0B
:107EE00023970FBEA20FB31F0FB66D962EAD3FADF9
:107EF0006D970FBE621E731E0FB62D962EAD3FAD51
:107F00002D970FBE0FB66B964EAD5FAD6B970FBE44
:107F1000242735276D857E852627372749895A8965
:107F200024273527B901660F771F0FB62B96EEADC4
:107F3000FFAD2B970FBE0FB667964EAD5FAD67973F
:107F40000FBEE427F5270FB661968EAC9FAC619704
:107F50000FBEE825F9250FB625964EAD5FAD2597E6
:107F60000FBEE427F527AF01452F42954F705527E7
:107F7000469546954695462B572B0FB627964EAFFE
:107F80005FAF27970FBEEE0FFF1F232F22952F7095
:107F900033272695269526952E2B3F2B0FB62D960B
:107FA0002EAF3FAF2D970FBEA40FB51FA301421FE9
:107FB000531FA80FB91F401F511FAA52BE434D495E
:107FC00055439D01BD010FB62B966EAF7FAF2B972A
:107FD0000FBE32952295307F3227207F3227220F25
:107FE000331FCA01DA01892F9927869586958695D0
:107FF000822B932B9D0132952295307F3227207F53
:108000003227220F331F672F77276695669566956F
:10801000622B732B96013695279536952795F70198
:10802000FE2FF295F07FEE27FF0FFF0FE22BF32BD1
:108030000FB66D96EEAFFFAF6D970FBE2D893E89DF
:10804000E227F3270FB665968EAC9FAC65970FBEFF
:10805000E825F925F694E794F694E7949601322FF3
:108060003295307F2227330F330F2E293F29890184
:10807000190129AE3AAE042515250A251B252FA581
:1080800038A94FA158A524273527CF84D8882C2577
:108090003D2549855A85242735273901220F331F6D
:1080A000EDA8FEA84D8D5E8DE426F5260FB62F9621
:1080B0004EAD5FAD2F970FBEE426F52649A95AA90C
:1080C000E426F526A701452F42954F705527469582
:1080D00046954695422B532B0FB629964EAF5FAF70
:1080E00029970FBEEE0CFF1C9301232F22952F70B2
:1080F00033272695269526952E293F292FA738AB7D
:108100000FB66996EEACFFAC69970FBEE40EF51E94
:108110004B895C89421F531F97012E0F3F1F401F41
:10812000511F280F391F461F571F2A523E434D49E2
:108130005543C901B9010FB669966EAF7FAF699714
:108140000FBE92958295907F9827807F9827880F01
:10815000991FFA016A01EF2FFF27E695E695E6954C
:10816000E82BF92B960132952295307F3227207F1C
:108170003227220F331F672F7727669566956695FE
:10818000622B732BC4019C01369527953695279554
:10819000A501542F5295507F4427550F550F422B60
:1081A000532B8A012A014DAA5EAA0FB66D962EADF9
:1081B0003FAD6D970FBE022713270FB62B968EACDF
:1081C0009FAC2B970FBE08251925B694A794B6949B
:1081D000A794982F9295907F8827990F990F8A29B5
:1081E0009B290FB665968EAF9FAF65970FBE7C013A
:1081F000E224F324EA26FB260FB66B964EAD5FAD64
:108200006B970FBE8DA59EA5482759276B8C7C8C3C
:10821000462557258B859C85482759279A01220F8B
:10822000331F0FB66796AEACBFAC67970FBE0FB6E5
:1082300063968EAD9FAD63970FBEA826B9262BAC73
:108240003CACA224B3248DA19EA1A826B926C501C9
:10825000892F82958F709927869586958695822B92
:10826000932B0FB623968EAF9FAF23970FBEAA0C0A
:10827000BB1C452F42954F70552746954695469510
:108280004A295B290FB66B964EAF5FAF6B970FBE57
:108290002D893E89280F391F8FA998AD841F951FFE
:1082A000200F311F8E1D9F1D2E0F3F1F861F971FF2
:1082B0002A523E438D4995437C01C901929582958E
:1082C000907F9827807F9827880F991FF701EF2FBD
:1082D000FF27E695E695E695E82BF92BC7019295E1
:1082E0008295907F9827807F9827880F991F890112
:1082F0001901012F1127069506950695082B192BB4
:10830000A401CA0196958795969587959D01322F70
:108310003295307F2227330F330F282B392BC90199
:1083200049010FB667968EAE9FAE67970FBE842544
:1083300095250FB669964EAC5FAC69970FBE842544
:108340009525B695A795B695A7959A01322F3295A2
:10835000307F2227330F330F2A2B3B2BA9013A0101
:108360000FB62B966EAE7FAE2B970FBE0FB66596EF
:108370004EAD5FAD65970FBE242735272C253D25D3
:108380008E0F9F1F201F311FEFA1F8A5498D5A8D19
:10839000E427F5274F8D58A1E427F5270FB6279638
:1083A0004EAD5FAD27970FBEE427F527AF01DF0184
:1083B000440F551FED8DFE8D6BA97CA9E627F7278D
:1083C0006DAD7EADE627F7270FB62D966EAD7FAD6E
:1083D0002D970FBEE627F727BF01672F62956F70B5
:1083E0007727669566956695642B752B6FAB78AF8E
:1083F000EE0FFF1FAB2FA295AF70BB27A695A695DA
:10840000A695AE2BBF2BAFA3B8A70FB66D964EADFA
:108410005FAD6D970FBE460F571F69AD7AAD6A1FEE
:108420007B1F480F591F621F731F4A525E436D49DD
:1084300075439A018A010FB66D960EAF1FAF6D9707
:108440000FBE32952295307F3227207F3227220FB0
:10845000331FCB015B01892F9927869586958695D9
:10846000822B932B950132952295307F3227207FE6
:108470003227220F331F012F1127069506950695E7
:10848000022B132BF201AF01569547955695479550
:10849000B601762F7295707F6627770F770F642B62
:1084A000752B9B012B014D8A5E8A282539254101B8
:1084B00028253925D694C794D694C794AF01542F54
:1084C0005295507F4427550F550F4C295D296A015D
:1084D0001A010FB669962EAE3FAE69970FBEC6243D
:1084E000D724CE24DF244DA95EA9240F351F0FB653
:1084F00065964EAD5FAD65970FBEC41ED51EEDA54A
:10850000FEA54F89588DE427F5270FB621964EAD6D
:108510005FAD21970FBEE427F5270FB629964EAD24
:108520005FAD29970FBEE427F527AF01440F551F14
:108530000FB663966EAD7FAD63970FBEABA5BCA5BE
:108540006A277B27A9A1BAA16A277B27AFA5B8A96B
:108550006A277B27DB01AB2FA295AF70BB27A695BF
:10856000A695A695A42BB52BAD8FBE8F660F771F52
:10857000EF2FE295EF70FF27E695E695E695E62B5F
:10858000F72BEDA7FEA72A0F3B1FD601AE1FBF1F7B
:10859000280F391FA01FB11F2A523E43AD49B543D2
:1085A000A9010FB665962EAF3FAF65970FBE5295E6
:1085B0004295507F5427407F5427440F551FCD01CB
:1085C0003D01892F9927869586958695842B952B35
:1085D000A30152954295507F5427407F5427440F62
:1085E000551FB901672F7727669566956695642BA9
:1085F000752BA4015695479556954795D701BA2FE7
:10860000B295B07FAA27BB0FBB0FA42BB52BA9AF88
:10861000BAAFA425B5250FB66D962EAD3FAD6D97BB
:108620000FBEA227B327F694E794F694E794A4012B
:10863000542F5295507F4427550F550F4E295F29CF
:108640008A012A01022513250A251B25E98DFA8DA9
:108650004BA15CA1E427F52749895A89E427F5272E
:108660000FB623964EAD5FAD23970FBEE427F527D7
:10867000AF014F01440F551F2BA83CA8E9A5FAA54F
:108680002E263F260FB62596CEACDFAC25970FBE23
:108690002C243D240FB66B96EEACFFAC6B970FBE4F
:1086A0002E243F24F101EF2FE295EF70FF27E6958E
:1086B000E695E695E42BF52BEDABFEAB220C331CD7
:1086C000A401452F42954F705527469546954695EE
:1086D000422953297A01E98EFA8E0FB667964EAD7C
:1086E0005FAD67970FBE4E0F5F1F0FB62B96EEADB7
:1086F000FFAD2B970FBEEE1DFF1D4A0F5B1FE01F46
:10870000F11F480F591FE61FF71F4A525E43ED49FC
:10871000F543BA01DA010FB66796AEAFBFAF679700
:108720000FBE72956295707F7627607F7627660F01
:10873000771FCF016F01892F99278695869586959A
:10874000862B972BA60152954295507F5427407F48
:108750005427440F551FBD01672F772766956695EF
:108760006695642B752B8901A801569547955695FA
:108770004795D501BA2FB295B07FAA27BB0FBB0F83
:10878000A42BB52B0FB62B96AEAFBFAF2B970FBE5A
:1087900029AD3AADA227B3270FB665962EAD3FADF2
:1087A00065970FBEA227B327B694A794B694A79453
:1087B000102F1295107F0027110F110F0A291B2966
:1087C0000FB66D960EAF1FAF6D970FBE0425152522
:1087D000120106251725EF89F88D2D853E85E227A4
:1087E000F32749855A85E427F5272FA938ADE227D5
:1087F000F327AF017F01440F551FABA4BCA40FB6F4
:1088000061962EAD3FAD61970FBEA226B32649A853
:108810005AA8A424B5242FA138A5A226B326F50171
:10882000EF2FE295EF70FF27E695E695E695E42BAE
:10883000F52B4F018FAA98AEAA0CBB1CA701452FA0
:1088400042954F7055274695469546954A295B298E
:108850007A01EF8AF88EED89FE89E80DF91D0FB6D1
:1088600069964EAD5FAD69970FBE4E1D5F1DEA0F55
:10887000FB1F401F511FE80FF91F461F571FEA52E9
:10888000FE434D495543CF014F01969587959695E7
:108890008795BA019A01762F7295707F6627770FB8
:1088A000770F682B792B6BA77CA7C90196958795C5
:1088B00096958795D401BA2FB295B07FAA27BB0FA2
:1088C000BB0FA82BB92BA9ABBAABE981FA81808980
:1088D000918942895389860F971F4A1F5B1F808B9E
:1088E000918B428B538B8F01C40192958295907F1F
:1088F0009827807F9827880F991F0FB669962EAF0B
:108900003FAF69970FBEB901672F772766956695C8
:108910006695682B792BC90192958295907F98274F
:10892000807F9827880F991FD401AB2FBB27A6956E
:10893000A695A695A82BB92B0FB665962EAD3FAD83
:1089400065970FBEC9019695879596958795A30162
:10895000542F5295507F4427550F550F482B592BB4
:108960000FB663964EAF5FAF63970FBECA010FB6E7
:108970002B964EAD5FAD2B970FBE842795270FB674
:108980006796EEACFFAC67970FBE8E259F25769459
:10899000679476946794322F3295307F2227330F75
:1089A000330F26293729F90139010FB665966EAEC6
:1089B0007FAE65970FBE0FB66D962EAD3FAD6D972E
:1089C0000FBEE227F327EC25FD25860F971FEA1F30
:1089D000FB1F6BA17CA12F853889622773272B850C
:1089E0003C85622773272D8D3E8D62277327AB014F
:1089F000440F551F29A53AA50FB62F96AEADBFADB2
:108A00002F970FBE2A273B27ADA1BEA12A273B27C0
:108A1000ADA5BEA52A273B27D901AB2FA295AF70E4
:108A2000BB27A695A695A695A42BB52BABABBCAB47
:108A3000220F331F672F62956F70772766956695B3
:108A40006695622B732B6BA37CA329AD3AAD2A0FDD
:108A50003B1FA101461F571F280F391F4E1F5F1FC5
:108A60002A523E434D495543C901290196958795A0
:108A7000969587959A011A01322F3295307F2227D9
:108A8000330F330F282B392BB9016DA77EA7C101F6
:108A900096958795969587959201322F3295307FDE
:108AA0002227330F330F282B392B29AF3AAFF80188
:108AB0008485958546855785860F971F421F531FCE
:108AC0008487958746875787C20192958295907FC4
:108AD0009827807F9827880F991FB101672F7727E4
:108AE000669566956695682B792BC101929582955E
:108AF000907F9827807F9827880F991F8201012FE8
:108B00001127069506950695082B192B9701C90183
:108B10009695879596958795A601542F5295507FE7
:108B20004427550F550F482B592B0FB625964EAF9E
:108B30005FAF25970FBE7A010FB663968EAD9FADDE
:108B400063970FBEE826F926E824F924D694C79443
:108B5000D694C794A901542F5295507F4427550F9E
:108B6000550F4C295D290FB667964EAF5FAF6797DB
:108B70000FBE462557250FB669968EAD9FAD6997F6
:108B80000FBE482759270FB62B968EAD9FAD2B975A
:108B90000FBEE80EF91E0FB66D968EAD9FAD6D97A8
:108BA0000FBE481F591FAD85BE858B8D9C8DA82794
:108BB000B9270FB627968EAD9FAD27970FBEA82772
:108BC000B9278DA99EA9A827B927CD01880F991F7C
:108BD0000FB661968EAC9FAC61970FBE2BAD3CADCE
:108BE000822693260FB62D962EAD3FAD2D970FBE44
:108BF00082269326298D3A8D822693269401232F4F
:108C000022952F703327269526952695282B392BCC
:108C1000880C991CAB2FA295AF70BB27A695A69583
:108C2000A695A829B9292E0D3F1DA41FB51F260FF3
:108C3000371FA01FB11F2A523E43AD49B543C9019A
:108C40009695879596958795AD01542F5295507FAF
:108C50004427550F550F482B592BCD0196958795D5
:108C600096958795B901762F7295707F6627770F55
:108C7000770F682B792B8085918502851385840F6A
:108C8000951F061F171F80879187028713875F0133
:108C9000C90192958295907F9827807F9827880FA9
:108CA000991FBD01672F7727669566956695682B96
:108CB000792BCD0192958295907F9827807F982778
:108CC000880F991FF901EF2FFF27E695E695E695A6
:108CD000E82BF92B6BA47CA473010FB625968EADFF
:108CE0009FAD25970FBEE826F926E424F52449A870
:108CF0005AA862010FB667968EAD9FAD67970FBEFB
:108D0000C826D926C224D3240F8D18A18F8598890F
:108D1000082719270FB629968EAD9FAD29970FBE4C
:108D2000082719278FA998AD08271927C801880F88
:108D3000991F8DAC9EAC0FB62F964EAD5FAD2F97A1
:108D40000FBE842695264FA558A9842695264F89BF
:108D5000588D84269526A401452F42954F7055279E
:108D6000469546954695482B592B880C991C012F02
:108D700002950F7011270695069506950829192961
:108D80000FB663968EAD9FAD63970FBE480F591F08
:108D90000FB665968EAD9FAD65970FBE081F191F64
:108DA0004E0D5F1D0C1D1D1D460F571F0E1F1F1F53
:108DB0004A525E430D491543F501848195816681D0
:108DC0007781840F951F601F711F8483958366834D
:108DD00077836F01CA0192958295907F9827807F53
:108DE0009827880F991FB801672F77276695669592
:108DF0006695682B792B12950295107F1027007FBE
:108E00001027000F111F452F55274695469546956B
:108E1000402B512B8DA59EA586259725822793272C
:108E20008C0189AD9AAD842595258A279B277C01E5
:108E30000FB62196AEADBFAD21970FBE8B8D9C8D29
:108E4000A827B9270FB623968EAD9FAD23970FBEE7
:108E5000A827B9278BA99CA9A827B927CD01880FD6
:108E6000991FE9A1FAA12BAD3CADE227F3270FB67C
:108E70006B962EAD3FAD6B970FBEE227F3272BA16C
:108E80003CA1E227F3279F01232F22952F70332740
:108E9000269526952695282B392BEE0FFF1FAB2FF5
:108EA000A295AF70BB27A695A695A695AE2BBF2B16
:108EB0000FB625968EAD9FAD25970FBE280F391F93
:108EC0000FB667968EAD9FAD67970FBEA81FB91FEF
:108ED000200F311FAE1DBF1D8B819C81280F391FB4
:108EE0008D819E81A81FB91F260F371FA41FB51F94
:108EF0002A523E43AD49B543F601A283B383208392
:108F00003183C456DF4F0FB6F894DEBF0FBECDBF1E
:108F1000DF91CF911F910F91FF90EF90DF90CF9055
:108F2000BF90AF909F908F907F906F905F904F9089
:108F30003F902F900895AA1BBB1B51E107C0AA1FA9
:108F4000BB1FA617B70710F0A61BB70B881F991FEA
:108F50005A95A9F780959095BC01CD01089581E0BF
:108F600090E0F8940C94D147FB01DC0104C08D9192
:108F70000190801921F441505040C8F7881B990B8B
:108F80000895FB01DC0102C001900D924150504058
:108F9000D8F70895DC0101C06D9341505040E0F7CF
:068FA0000895F894FFCFD4
:108FA600530004000100AE0E53000000010037100C
:108FB6005300020001001E092509CE0953000600D0
:108FC60001002B054208E808303132333435363794
:108FD6003839616263646566486F6C61206D756ED1
:108FE600646F3078303030313032303330343035B1
:108FF6003036303730383039313031313132313343
:109006003134313531363137313831393230323128
:10901600323232333234323532363237323832390E
:109026003330333133323333333433353336333706
:1090360033383339343034313432343334343435EC
:1090460034363437343834393530353135323533D2
:1090560035343535353635373538353936303631B8
:10906600363236333634363536363637363836399E
:109076003730373137323733373437353736373796
:10908600373837393830383138323833383438357C
:109096003836383738383839393039313932393362
:1090A600393439353936393739383939536F6D6589
:1090B6004E6F6E6520202020010101010101010192
:1090C600010101010101010101010101010101018A
:1090D600010101010101010101010101010101017A
:1090E600010101010101010101010101010101016A
:1090F600010101010101010101010101010101015A
:109106000101010101010101010101010101010149
:109116000101010101010101010101010101010139
:109126000101010101010101010101010101010129
:109136000101010101010101000000000000000021
:109146000000000000000000000000000000000019
:109156000000000000000000000000000000000009
:1091660000000000000000000000000000000000F9
:1091760000000000000000000000020202020202DD
:1091860002020202020202020202020202020202B9
:1091960002020202020202020303030303030303A1
:1091A600030303030303030304040404040000008D
:1091B6000000000000000000207B0A3A202C0A2C48
:1091C60020207B207D207D280A2829557466384575
:1091D60072726F7276616C69645F75705F746F65C9
:1091E60072726F725F6C656E576F756C64426C6FEE
:1091F600636B0123456789ABCDEFFEDCBA987654E5
:069206003210F0E1D2C3BA
:00000001FF
